:020000040800F2
:1000000000800020016600081D1200081F12000871
:100010002112000823120008251200080000000029
:10002000000000000000000000000000271200088F
:1000300029120008000000002B1200082D120008F1
:1000400051660008516600085166000851660008B4
:1000500051660008516600085166000851660008A4
:100060005166000851660008516600085166000894
:1000700035120008451200085512000851660008A4
:100080005166000800000000651200085166000873
:100090005166000851660008516600085166000864
:1000A0005166000851660008516600085166000854
:1000B0007D120008AD120008516600085166000864
:1000C0005166000851660008516600085166000834
:1000D00051660008C5120008516600085166000804
:1000E0005166000851660008516600085166000814
:1000F00051660008516600085166000800000000C3
:100100000000000051660008000000005166000871
:1001100051660008000000005166000851660008A2
:1001200051660008516600085166000851660008D3
:100130005166000800000000000000005166000841
:100140005166000851660008000000000000000031
:10015000000000000000000000000000000000009F
:1001600000000000000000000000000051660008D0
:1001700051660008000000000000000000000000C0
:1001800000000000516600080000000000000000B0
:10019000000000000000000000000000000000005F
:1001A00000000000000000005166000851660008D1
:1001B0005166000851660008516600080000000002
:1001C0000000000051660008000000000000000070
:0801D0005166000851660008A9
:1001E000034613F8012B002AFBD1181A0138704777
:1001F00001F0FF01102A2BDB10F0070F08D010F8D8
:10020000013B013A8B422DD010F0070F42B3F6D1DB
:10021000F0B441EA012141EA014122F007047FF0F4
:1002200000070023F0E80256083C85EA010586EA4B
:10023000010685FA47F5A3FA87F586FA47F6A5FA87
:1002400087F68EB9EED1F0BC01F0FF0102F0070293
:1002500032B110F8013B013A83EA010313B1F8D13E
:100260000020704701387047002D06BF354603381F
:10027000073815F0010F07D1013015F4807F02BF58
:10028000013015F4C03F0130F0BC0138704700BFA9
:1002900081F0004102E000BF83F0004330B54FEA37
:1002A00041044FEA430594EA050F08BF90EA020FA4
:1002B0001FBF54EA000C55EA020C7FEA645C7FEA37
:1002C000655C00F0E2804FEA5454D4EB5555B8BF5A
:1002D0006D420CDD2C4480EA020281EA030382EACB
:1002E000000083EA010180EA020281EA0303362D5D
:1002F00088BF30BD11F0004F4FEA01314FF4801C30
:100300004CEA113102D0404261EB410113F0004F41
:100310004FEA03334CEA133302D0524263EB4303F8
:1003200094EA050F00F0A780A4F10104D5F1200E96
:100330000DDB02FA0EFC22FA05F2801841F10001F1
:1003400003FA0EF2801843FA05F359410EE0A5F1C5
:1003500020050EF1200E012A03FA0EFC28BF4CF0F6
:10036000020C43FA05F3C01851EBE37101F00045AC
:1003700007D54FF0000EDCF1000C7EEB00006EEBB9
:100380000101B1F5801F1BD3B1F5001F0CD3490843
:100390005FEA30004FEA3C0C04F101044FEA44529A
:1003A00012F5800F80F09A80BCF1004F08BF5FEA21
:1003B000500C50F1000041EB045141EA050130BD01
:1003C0005FEA4C0C404141EB0101013C28BFB1F513
:1003D000801FE9D291F0000F04BF01460020B1FA5E
:1003E00081F308BF2033A3F10B03B3F120020CDA31
:1003F0000C3208DD02F1140CC2F10C0201FA0CF00F
:1004000021FA02F10CE002F11402D8BFC2F1200C73
:1004100001FA02F120FA0CFCDCBF41EA0C01904029
:10042000E41AA2BF01EB0451294330BD6FEA040472
:100430001F3C1CDA0C340EDC04F11404C4F120025D
:1004400020FA04F001FA02F340EA030021FA04F36F
:1004500045EA030130BDC4F10C04C4F1200220FAC6
:1004600002F001FA04F340EA0300294630BD21FA04
:1004700004F0294630BD94F0000F83F4801306BFCA
:1004800081F480110134013D4EE77FEA645C18BFBE
:100490007FEA655C29D094EA050F08BF90EA020F55
:1004A00005D054EA000C04BF1946104630BD91EA4D
:1004B000030F1EBF0021002030BD5FEA545C05D150
:1004C0004000494128BF41F0004130BD14F580048F
:1004D0003CBF01F5801130BD01F0004545F0FE4103
:1004E00041F470014FF0000030BD7FEA645C1ABF38
:1004F000194610467FEA655C1CBF0B46024650EA6F
:10050000013406BF52EA033591EA030F41F400219A
:1005100030BD00BF90F0000F04BF0021704730B520
:100520004FF4806404F132044FF000054FF00001F5
:1005300050E700BF90F0000F04BF0021704730B5B6
:100540004FF4806404F1320410F0004548BF40428B
:100550004FF000013EE700BF42004FEAE2014FEAE0
:1005600031014FEA02701FBF12F07F4393F07F4FBB
:1005700081F06051704732F07F4208BF704793F0BE
:100580007F4F04BF41F40021704730B54FF46074D1
:1005900001F0004521F000411CE700BF50EA0102D4
:1005A00008BF704730B54FF000050AE050EA01027D
:1005B00008BF704730B511F0004502D5404261EBED
:1005C00041014FF4806404F132045FEA915C3FF42E
:1005D000D8AE4FF003025FEADC0C18BF03325FEACB
:1005E000DC0C18BF033202EBDC02C2F1200300FA7C
:1005F00003FC20FA02F001FA03FE40EA0E0021FAA1
:1006000002F11444BDE600BF70B54FF0FF0C4CF48E
:10061000E06C1CEA11541DBF1CEA135594EA0C0F40
:1006200095EA0C0F00F0DEF82C4481EA030621EA7B
:100630004C5123EA4C5350EA013518BF52EA0335B6
:1006400041F4801143F4801338D0A0FB02CE4FF068
:100650000005E1FB02E506F00042E0FB03E54FF098
:100660000006E1FB03569CF0000F18BF4EF0010E90
:10067000A4F1FF04B6F5007F64F5407404D25FEA8C
:100680004E0E6D4146EB060642EAC62141EA55513F
:100690004FEAC52040EA5E504FEACE2EB4F1FD0C81
:1006A00088BFBCF5E06F1ED8BEF1004F08BF5FEAFF
:1006B000500E50F1000041EB045170BD06F00046B1
:1006C00046EA010140EA020081EA0301B4EB5C045E
:1006D000C2BFD4EB0C0541EA045170BD41F4801156
:1006E0004FF0000E013C00F3AB8014F1360FDEBF7B
:1006F000002001F0004170BDC4F10004203C35DA57
:100700000C341BDC04F11404C4F1200500FA05F3D9
:1007100020FA04F001FA05F240EA020001F000427A
:1007200021F0004110EBD37021FA04F642EB0601F0
:100730005EEA430E08BF20EAD37070BDC4F10C041A
:10074000C4F1200500FA04F320FA05F001FA04F2DE
:1007500040EA020001F0004110EBD37041F10001CA
:100760005EEA430E08BF20EAD37070BDC4F12005D5
:1007700000FA05F24EEA020E20FA04F301FA05F23D
:1007800043EA020321FA04F001F0004121FA04F2E5
:1007900020EA020000EBD3705EEA430E08BF20EAB5
:1007A000D37070BD94F0000F0FD101F000464000EF
:1007B00041EB010111F4801F08BF013CF7D041EA71
:1007C000060195F0000F18BF704703F00046520075
:1007D00043EB030313F4801F08BF013DF7D043EA46
:1007E0000603704794EA0C0F0CEA135518BF95EAFC
:1007F0000C0F0CD050EA410618BF52EA4306D1D183
:1008000081EA030101F000414FF0000070BD50EAA1
:10081000410606BF1046194652EA430619D094EA2B
:100820000C0F02D150EA013613D195EA0C0F05D115
:1008300052EA03361CBF104619460AD181EA030169
:1008400001F0004141F0FE4141F470014FF0000021
:1008500070BD41F0FE4141F4780170BD70B54FF0BC
:10086000FF0C4CF4E06C1CEA11541DBF1CEA13553C
:1008700094EA0C0F95EA0C0F00F0A7F8A4EB05041E
:1008800081EA030E52EA03354FEA013100F0888015
:100890004FEA03334FF0805545EA131343EA1263DE
:1008A0004FEA022245EA111545EA10654FEA002693
:1008B0000EF000419D4208BF964244F1FD0404F54C
:1008C000407402D25B084FEA3202B61A65EB0305A8
:1008D0005B084FEA32024FF480104FF4002CB6EB65
:1008E000020E75EB030E22BFB61A754640EA0C00E5
:1008F0005B084FEA3202B6EB020E75EB030E22BF25
:10090000B61A754640EA5C005B084FEA3202B6EB65
:10091000020E75EB030E22BFB61A754640EA9C0024
:100920005B084FEA3202B6EB020E75EB030E22BFF4
:10093000B61A754640EADC0055EA060E18D04FEAB2
:10094000051545EA16754FEA06164FEAC30343EA52
:1009500052734FEAC2025FEA1C1CC0D111F4801F1F
:100960000BD141EA00014FF000004FF0004CB6E718
:1009700011F4801F04BF01430020B4F1FD0C88BFB7
:10098000BCF5E06F3FF6AFAEB5EB030C04BFB6EBC2
:10099000020C5FEA500C50F1000041EB045170BDB5
:1009A0000EF0004E4EEA113114EB5C04C2BFD4EBE2
:1009B0000C0541EA045170BD41F480114FF0000E66
:1009C000013C90E645EA060E8DE60CEA135594EAE2
:1009D0000C0F08BF95EA0C0F3FF43BAF94EA0C0FE5
:1009E0000AD150EA01347FF434AF95EA0C0F7FF45A
:1009F00025AF104619462CE795EA0C0F06D152EAAE
:100A000003353FF4FDAE1046194622E750EA410691
:100A100018BF52EA43067FF4C5AE50EA41047FF4A2
:100A20000DAF52EA43057FF4EBAE12E74FEA410205
:100A300012F5001215D211D56FF47873B3EB625230
:100A400012D94FEAC12343F0004343EA505311F057
:100A5000004F23FA02F018BF404270474FF00000E9
:100A6000704750EA013005D111F0004008BF6FF027
:100A7000004070474FF00000704700BF4A0011D29D
:100A800012F5001211D20DD56FF47873B3EB6252E8
:100A90000ED44FEAC12343F0004343EA505323FAF4
:100AA00002F070474FF00000704750EA013002D169
:100AB0004FF0FF3070474FF00000704753B94AB90C
:100AC000002908BF00281CBF4FF0FF314FF0FF3056
:100AD00000F00CB8ADF1080C6DE904CE06F06EFA2A
:100AE000DDF804E0DDE9022304B07047704700BF81
:100AF0000348044B834202D0034B03B118477047AD
:100B00005C0000205C000020000000000548064B4F
:100B10001B1AD90F01EBA301491002D0034B03B1FB
:100B2000184770475C0000205C00002000000000B7
:100B300010B5064C237843B9FFF7DAFF044B13B125
:100B40000448AFF300800123237010BD6000002033
:100B5000000000007872000808B5054B1BB105497C
:100B60000548AFF30080BDE80840FFF7CFBF00BFE6
:100B700000000000640000207872000830B58BB0DF
:100B8000002405940694079408940994214BDA6C88
:100B900042F02002DA64DA6C02F020020192019A3B
:100BA000DA6C42F04002DA64DA6C02F0400202923F
:100BB000029ADA6C42F00102DA64DA6C02F00102A5
:100BC0000392039ADA6C42F00202DA64DB6C03F0FF
:100BD00002030493049B104D22467821284601F01D
:100BE00061FC4FF4806305930223069307940894F5
:100BF000099405A9094801F06BFB782305930123AB
:100C000006930794089405A9284601F061FB0BB0F0
:100C100030BD00BF0010024000040048001800482A
:100C200000B583B0164B9A6C42F004029A649A6C39
:100C300002F004020092009A9A6C42F001029A6457
:100C40009B6C03F001030193019B002211460C20D1
:100C500001F0F4FE0C2001F001FF002211460D20EE
:100C600001F0ECFE0D2001F0F9FE002211460E20ED
:100C700001F0E4FE0E2001F0F1FE03B05DF804FB8C
:100C80000010024070470000014B01221A707047AB
:100C900018040020084B1B888B420BD006D9064B4A
:100CA00000221A8002E00133034A1380024B1B88A2
:100CB0008B42F8D3704700BF7C000020014B01221B
:100CC0001A7070476A04002072B6FEE700B58FB054
:100CD00000230A930B930C930D93079308930993A6
:100CE000009301930293039304930593069333486F
:100CF0004FF0804202604360836040F6FF72C26042
:100D00000361836103F0AAFF002846D14FF48053AA
:100D10000A930AA9294804F0F1F800283FD127488E
:100D200003F0CCFF00283CD1202307930023099334
:100D300007A9224804F03EFA002834D1602300932A
:100D40004FF4FA730193002202920423049369463C
:100D50001A4804F029F840BB4FF47A730193042237
:100D60006946164804F020F808BB40F2DC530193B2
:100D700008226946114804F017F8D0B94FF4FA6315
:100D800001930C2269460D4804F00EF898B90B48FF
:100D900000F002FC0FB05DF804FBFFF795FFFFF7D2
:100DA00093FFFFF791FFFFF78FFFFFF78DFFFFF72F
:100DB0008BFFFFF789FFFFF787FF00BF20020020AE
:100DC00008B51148114B0360114B43600023836049
:100DD0000122C260036143618361C361036203F066
:100DE0001AF950B90021084803F0C5FB38B90021B1
:100DF000054803F0EEFB20B908BDFFF765FFFFF7DC
:100E000063FFFFF761FF00BF6C0200200054004049
:100E1000BD82B24000B589B00023049305930693C8
:100E200007930193029303931348144A02604AF212
:100E3000FF124260836040F28F12C26003618361DF
:100E400003F00CFF90B94FF48053049304A90A48AF
:100E500004F054F860B900230193039301A90648F4
:100E600004F0A8F930B909B05DF804FBFFF72CFFD6
:100E7000FFF72AFFFFF728FFD401002000040040FD
:100E800010B592B000240F94109411940894099412
:100E90000A940B940C940D940E94202221466846DB
:100EA00005F002FC2C484FF0A04303604FF44033A0
:100EB00043608460C46004614461042383610477F7
:100EC00044770123036280F824404FF4AC63C3628B
:100ED0004FF48063036380F83840C46380F8404077
:100EE00001F01AFE00282FD100230F930FA91A48F2
:100EF00002F036FE50BB194B08934FF440030993A0
:100F0000174B0A9301238DF82C304FF47D630C931B
:100F100030230D9300230E9308A90F4802F0EAFA3C
:100F2000B0B90F4B009306230193052302937F234F
:100F3000039304230493002305936946064802F0B3
:100F4000A9F838B912B010BDFFF7BEFEFFF7BCFE1E
:100F5000FFF7BAFEFFF7B8FE8C0300200000C07D4B
:100F60000080F03E00B589B020220021684605F0DF
:100F70009BFB2B482B4B03604FF440334360002313
:100F80008360C360036101224261082282610377AA
:100F900043770422026280F82430C362036380F83E
:100FA0003830C36380F8403001F0B6FD00282DD101
:100FB0001D4B00930623019302937F230393042385
:100FC0000493002305936946154802F063F8F8B9C5
:100FD000164B00930C2301936946114802F05AF80E
:100FE000C0B9134B00931223019369460C4802F0D9
:100FF00051F888B90F4B00931823019369460848AC
:1010000002F048F850B909B05DF804FBFFF75CFE48
:10101000FFF75AFEFFF758FEFFF756FEFFF754FEA4
:1010200020030020000100500800900C1000C010A8
:10103000002090360000524708B51548154B036054
:101040004FF4E133436000238360C36003610C22EB
:1010500042618361C36103624362836204F0B6FE4E
:1010600070B900210A4804F085FF58B900210848EA
:1010700004F0A5FF40B9064804F05DFF30B908BD93
:10108000FFF722FEFFF720FEFFF71EFEFFF71CFE14
:10109000400100200038014000B595B03822002101
:1010A00006A805F001FB0020019002900390049037
:1010B000059001F0E1FB012306934FF48033079381
:1010C00002230D9303220E920F9336221092119356
:1010D00004221292139306A800F07EFBB0B90F23EE
:1010E00001930323029300230393049305930421A4
:1010F0000DEB010000F054FE50B900224FF080616A
:10110000044800F0DBFD15B05DF804FBFFF7DCFDE3
:10111000FFF7DAFD0004060008B500F00FFBFFF74B
:10112000BBFFFFF72BFDFFF77BFDFFF7CFFDFFF7C1
:1011300047FEFFF76FFEFFF7A3FEFFF713FFFFF772
:101140007BFF40222A492B4804F05EFF2A4802F028
:10115000B5FB2A4C204603F0DFFB294803F0DCFBFB
:101160000021204603F076FF0421204603F072FFA1
:101170000821204603F06EFF0C21204603F06AFF91
:1011800005F072F905F0E2F904221E491E4802F04A
:101190005DFC05F0B1F91D4805F0B8F905F0C8F996
:1011A0000FE004221749184802F050FC184B0022A7
:1011B0001A700EE0174A137801331370164B002291
:1011C0001A70154B1B78002BFBD0114B1B78002B92
:1011D000E7D1104B1B780A2BECD905F0D3F90D4B56
:1011E00000221A70094805F091F905F0A1F9E1E72C
:1011F00028040020400100208C0300202002002051
:10120000D40100201C0400202003002098BC1400FE
:10121000180400206804002069040020FEE7FEE7AF
:10122000FEE7FEE7FEE770477047704708B500F03D
:1012300095FA08BD08B5024801F0BBFA08BD00BF29
:10124000C002002008B5024801F0B3FA08BD00BF93
:10125000E000002008B5024801F0ABFA08BD00BF6D
:101260008000002008B5034801F074FD024801F039
:1012700071FD08BD8C0300202003002010B5084834
:1012800003F092FB074801F05BFD84B2204605F0B5
:101290001DF9054B18704FF080435C639C6310BDD3
:1012A000200200208C0300206D04002008B50348B4
:1012B00003F07AFB024B01221A7008BDD401002012
:1012C0006904002008B5024804F052F808BD00BFC8
:1012D0004001002000B583B00B4B1A6E42F00102B2
:1012E0001A661A6E02F001020092009A9A6D42F09C
:1012F00080529A659B6D03F080530193019B01F02E
:1013000041FB03B05DF804FB0010024030B59BB018
:1013100004460021159116911791189119914422B4
:1013200004A805F0C1F92368B3F1A04F04D04B4ADB
:1013300093423CD01BB030BD4FF4004304934FF0B8
:101340000053139304A800F051FE10BB444A1368E5
:1013500001331360012B1FD0424BDA6C42F00202C2
:10136000DA64DB6C03F002030193019B0123159304
:10137000032316930024179415A93B4800F0A8FFF7
:1013800022462146122001F059FB122001F066FB93
:10139000D0E7FFF799FCD9E7324BDA6C42F4005200
:1013A000DA64DB6C03F400530093009BD4E74FF442
:1013B000004304934FF00053139304A800F016FE6B
:1013C00000283AD1264A136801331360012B37D025
:1013D000244BDA6C42F00102DA64DB6C03F00103A7
:1013E0000393039BF023159303231693002517956E
:1013F00015A94FF0904000F06BFF1C481C4B036098
:10140000242343608560C560802303614FF48073AB
:1014100043614FF480638361C561056201F0A0F808
:10142000C8B9124B63659C6200221146122001F07C
:1014300005FB122001F012FB7CE7FFF745FCC1E73A
:10144000084BDA6C42F40052DA64DB6C03F40053AC
:101450000293029BBCE7FFF737FCE2E70001005074
:10146000F80300200010024000040048C0020020E1
:101470001C000240F0B59BB0044600211591169166
:10148000179118911991442204A805F00DF92268CA
:10149000224B9A4201D01BB0F0BD4023049304A814
:1014A00000F0A4FD002835D11D4CE36C43F001038E
:1014B000E364E36C03F001030193019BE36C43F0ED
:1014C0000203E364E36C03F002030293029B4FF414
:1014D0000043159312271697002517951895042693
:1014E000199615A94FF0904000F0F2FE8023159355
:1014F000169717951895199615A90A4800F0E8FE51
:10150000A36D43F40013A365A36D03F400130393C9
:10151000039BC0E7FFF7D8FBC6E700BF00540040BD
:10152000001002400004004800B583B00368B3F126
:10153000804F05D0164A934216D003B05DF804FBE5
:1015400003F504339A6D42F001029A659B6D03F036
:1015500001030093009B002211461C2001F06EFA4B
:101560001C2001F07BFAE8E70A4B9A6D42F0020278
:101570009A659B6D03F002030193019B00221146C3
:101580001D2001F05BFA1D2001F068FAD5E700BFCD
:10159000000400400010024000B587B00023019312
:1015A00002930393049305930368B3F1804F02D031
:1015B00007B05DF804FB03F50433DA6C42F0010276
:1015C000DA64DB6C03F001030093009B0F230193AB
:1015D000022302930123059301A94FF0904000F0EC
:1015E00077FEE5E730B599B00446002113911491D8
:1015F000159116911791442202A805F055F822681A
:10160000344B9A4201D019B030BD0123029302A895
:1016100000F0ECFC002853D12F4B1A6E42F48042AC
:101620001A661A6E02F480420092009ADA6C42F056
:101630000102DA64DB6C03F001030193019B4FF4B8
:10164000C063139302231493002515951693072363
:10165000179313A94FF0904000F03AFE1F48204B1B
:101660000360182343608560C56080230361456182
:101670008561C561056200F073FF20BB174BC4F89C
:1016800080309C621748184B036019234360102375
:1016900083600023C3608022026143618361C36170
:1016A000036200F05DFF88B90E4BE3679C62002285
:1016B0001146252001F0C2F9252001F0CFF9A2E75B
:1016C000FFF702FBA8E7FFF7FFFAD7E7FFF7FCFAFF
:1016D000EAE700BF0038014000100240E0000020AF
:1016E000300002408000002044000240104B1B6884
:1016F0000BB90120704710B504464FF47A70B0FB67
:10170000F3F30C4A1068B0FBF3F001F0ABF968B9E1
:101710000F2C01D901200AE0002221464FF0FF30B2
:1017200001F08CF9044B1C60002000E0012010BD8A
:1017300000000020080000200400002010B5032055
:1017400001F06AF90020FFF7D1FF10B10124204613
:1017500010BD0446FFF7BEFDF9E70000034A136819
:10176000034909680B441360704700BFFC03002065
:1017700000000020014B1868704700BFFC030020E8
:10178000124BDA6802F00302DB68C3F30313013380
:10179000032A11D00E48B0FBF3F00C4BDB68C3F307
:1017A000062303FB00F0094BDB68C3F341630133FD
:1017B0005B00B0FBF3F070470648B0FBF3F0034B5F
:1017C000DB68C3F3062303FB00F0ECE700100240E4
:1017D0000024F4000080BB00002800F04F8270B5A8
:1017E00082B00446036813F0010F37D0A44A93680F
:1017F00003F00C03D26802F003020C2B23D0082B59
:1018000023D06368B3F5803F4ED0B3F5A02F51D0FD
:101810009B4B1A6822F480321A601A6822F48022E4
:101820001A606368002B52D0FFF7A4FF0546944B63
:101830001B6813F4003F11D1FFF79CFF401B642885
:10184000F5D9032023E2032AD9D18D4B1B6813F469
:10185000003F03D06368002B00F01282236813F06E
:10186000020F5DD0864A936803F00C03D26802F041
:1018700003020C2B3AD0042B3AD0E368002B75D02E
:101880007F4A136843F480731360FFF773FF0546C4
:101890007B4B1B6813F4806F5FD1FFF76BFF401B1E
:1018A0000228F5D90320F2E1754A136843F4803326
:1018B0001360B6E703F18043A3F53C331A6842F4A2
:1018C00080221A601A6842F480321A60A9E7FFF792
:1018D00051FF05466A4B1B6813F4003FBED0FFF76B
:1018E00049FF401B6428F5D90320D0E1022AC2D168
:1018F000634B1B6813F4806F03D0E368002B00F088
:10190000C1815F4A536823F0FE43216943EA0163C2
:1019100053605C4B1868FFF7E9FE002840F0B48183
:10192000236813F0080F4CD063699BB3544AD2F874
:10193000943043F00103C2F89430FFF71BFF0546D3
:101940004F4BD3F8943013F0020F3AD1FFF712FF48
:10195000401B0228F4D9032099E1494A536823F037
:10196000FE43216943EA01635360D9E7444A13689F
:1019700023F480731360FFF7FDFE0546404B1B68A0
:1019800013F4806FCCD0FFF7F5FE401B0228F5D989
:1019900003207CE13A4AD2F8943023F00103C2F8E4
:1019A0009430FFF7E7FE0546354BD3F8943013F03B
:1019B000020F06D0FFF7DEFE401B0228F4D90320F9
:1019C00065E1236813F0040F00F081802C4B9B6DC0
:1019D00013F0805F36D12A4B9A6D42F080529A659F
:1019E0009B6D03F080530193019B0125264B1B68DF
:1019F00013F4807F28D0A368012B39D0052B45D064
:101A00001F4BD3F8902022F00102C3F89020D3F8A6
:101A1000902022F00402C3F89020A368002B43D04A
:101A2000FFF7A8FE0646164BD3F8903013F0020FCE
:101A30004CD1FFF79FFE801B41F288339842F2D9C8
:101A4000032024E10025D1E70F4A136843F4807393
:101A50001360FFF78FFE06460B4B1B6813F4807F65
:101A6000C9D1FFF787FE801B0228F5D903200EE1BC
:101A7000034AD2F8903043F00103C2F89030CCE72B
:101A8000001002400400002000700040884BD3F892
:101A9000902042F00402C3F89020D3F8902042F046
:101AA0000102C3F89020B8E7FFF764FE0646804BBA
:101AB000D3F8903013F0020F08D0FFF75BFE801BC5
:101AC00041F288339842F2D90320E0E0E5B9236877
:101AD00013F0200F35D0A369E3B1754AD2F89830DE
:101AE00043F00103C2F89830FFF744FE0546704BFF
:101AF000D3F8983013F0020F23D1FFF73BFE401BC1
:101B00000228F4D90320C2E0694A936D23F0805380
:101B10009365DCE7664AD2F8983023F00103C2F8F7
:101B20009830FFF727FE0546614BD3F8983013F045
:101B3000020F06D0FFF71EFE401B0228F4D9032037
:101B4000A5E0E369002B00F0A180594A926802F0F9
:101B50000C020C2A64D0022B13D0554A136823F0D0
:101B600080731360FFF706FE0446514B1B6813F0A9
:101B7000007F4ED0FFF7FEFD001B0228F5D90320A1
:101B800085E04B4A136823F080731360FFF7F2FD82
:101B90000546474B1B6813F0007F06D0FFF7EAFDB0
:101BA000401B0228F5D9032071E0414AD36841491E
:101BB0001940236A606A013843EA0013A06A43EAC5
:101BC0000023206B4008013843EA4053606B400813
:101BD000013843EA4063E06A43EAC0631943D160D5
:101BE000136843F080731360D36843F08073D3604D
:101BF000FFF7C0FD04462E4B1B6813F0007F06D193
:101C0000FFF7B8FD001B0228F5D903203FE00020B4
:101C10003DE0274AD168284B0B40D360002036E0D6
:101C2000012B36D0224BDB6803F00301226A91427C
:101C300031D103F0F002616A0139B2EB011F2CD1FE
:101C400003F4FE42A16AB2EB012F28D103F07842DF
:101C5000E16AB2EBC16F24D103F4C001226B5208D8
:101C6000013AB1EB425F1ED103F0C063626B5208D0
:101C7000013AB3EB426F18D1002008E00120704711
:101C8000012004E0012002E0012000E0002002B079
:101C900070BD0120FBE70120F9E70120F7E70120F3
:101CA000F5E70120F3E70120F1E70120EFE700BFAE
:101CB000001002400C809F01FCFFEEFE70B586B064
:101CC0000C46154602230293032304930023039337
:101CD00000F08056C0F3034C0CF5901E0D4AD36CF7
:101CE000012101FA0CF10B43D36483B20193C0F3D9
:101CF0000750059001A94FEA8E2000F0E9FA36B9A5
:101D0000044A936823F0FE432C431C43946006B0BE
:101D100070BD00BF001002401E4B9B6803F00C0317
:101D2000042B33D01B4B9B6803F00C03082B2FD0E4
:101D3000184B9B6803F00C030C2B01D0002070475C
:101D4000144BDA6802F00302DB68C3F303130133B8
:101D5000032A11D01048B0FBF3F00E4BDB68C3F33D
:101D6000062303FB00F00B4BDB68C3F34163013335
:101D70005B00B0FBF3F070470848B0FBF3F0054B95
:101D8000DB68C3F3062303FB00F0ECE7024870476F
:101D900002487047001002400024F4000080BB009D
:101DA000002800F0E680F8B50C460546744B1B6829
:101DB00003F00F038B420BD2714A136823F00F0319
:101DC0000B431360136803F00F038B4240F0D38082
:101DD0002E6816F001065FD06B68032B2FD0022B04
:101DE0004DD0684B1B6813F4806F00F0C680FFF77E
:101DF00093FF654B98424DD9624A936823F0F003F4
:101E000043F08003936080265E4A936823F00303C7
:101E100069680B439360FFF7ADFC0746594B9B681D
:101E200003F00C036A68B3EB820F35D0FFF7A2FC16
:101E3000C01B41F288339842F0D9032078E0514B1F
:101E40001B6813F0007F01D1012071E0FFF798FCBF
:101E50004D4B98421AD94B4B9B6813F0F00F05D0AD
:101E60002E6816F00206CFD0AB688BB9454A93684E
:101E700023F0F00343F0800393608026C4E7414BD6
:101E80001B6813F4003FB2D1012051E00026BBE7EC
:101E90000026B9E70026B7E72B6813F0020F48D0F9
:101EA00013F0040F04D0374A936843F4E06393605F
:101EB0002B6813F0080F06D0324A936823F47C5342
:101EC00043F4E06393602F4A936823F0F003A9681A
:101ED0000B4393602A4B1B6803F00F03A34230D8D7
:101EE0002B6813F0040F06D0264A936823F4E063AE
:101EF000E9680B4393602B6813F0080F07D0214A61
:101F0000936823F46053296943EAC1039360FFF7A0
:101F100003FF1C4B9B68C3F303131C4AD35C03F001
:101F20001F03D8401A4B18601A4B1868FFF7DEFBE6
:101F3000F8BD802ECED1134A936823F0F00393604E
:101F4000C8E70F4A136823F00F0323431360FFF71A
:101F500011FC06460A4B1B6803F00F03A342BFD0D7
:101F6000FFF708FC801B41F288339842F2D9032026
:101F7000DEE7012070470120DAE70120D8E700BF43
:101F8000002002400010024000B4C404C0720008E7
:101F90000800002004000020014B1868704700BFB3
:101FA0000800002008B5FFF7F7FF054B9B68C3F357
:101FB0000223044AD35C03F01F03D84008BD00BFCE
:101FC00000100240B872000808B5FFF7E5FF054BA6
:101FD0009B68C3F3C223044AD35C03F01F03D840B9
:101FE00008BD00BF00100240B8720008F0B583B011
:101FF0000446036813F4002F69D0AE4B9B6D13F0B9
:10200000805F1ED1AB4B9A6D42F080529A659B6DFA
:1020100003F080530193019B0126A74A136843F400
:1020200080731360FFF7A6FB0546A34B1B6813F4F0
:10203000807F08D1FFF79EFB401B0228F5D90325BE
:1020400002E00026E9E7002545BB9A4BD3F8903023
:1020500013F4407315D0226C9A4212D0954AD2F8EC
:10206000903023F44073D2F8901041F48031C2F8DC
:102070009010D2F8901021F48031C2F89010C2F87C
:10208000903013F0010F10D145B98A4AD2F8903040
:1020900023F44073216C0B43C2F89030C6B1854ADB
:1020A000936D23F08053936512E0FFF763FB0746BF
:1020B000804BD3F8903013F0020FE5D1FFF75AFBB5
:1020C000C01B41F288339842F2D90325DCE7002592
:1020D000236813F0010F08D0764AD2F8883023F035
:1020E000030361680B43C2F88830236813F0020FC2
:1020F00008D0704AD2F8883023F00C03A1680B4353
:10210000C2F88830236813F0040F08D0694AD2F867
:10211000883023F03003E1680B43C2F8883023682D
:1021200013F0080F08D0634AD2F8883023F0C003B8
:1021300021690B43C2F88830236813F0200F08D0C0
:102140005C4AD2F8883023F4406361690B43C2F8DB
:102150008830236813F0400F08D0564AD2F88830F0
:1021600023F44053A1690B43C2F88830236813F06D
:10217000800F08D04F4AD2F8883023F44043E169F9
:102180000B43C2F88830236813F4807F08D0494A93
:10219000D2F8883023F44033216A0B43C2F88830E8
:1021A000236813F4007F08D0424AD2F8883023F421
:1021B0004023616A0B43C2F88830236813F4806FB0
:1021C0000CD03C4AD2F8883023F44013A16A0B4368
:1021D000C2F88830A36AB3F5801F57D0236813F480
:1021E000006F0CD0334AD2F8883023F44003E16A00
:1021F0000B43C2F88830E36AB3F5800F4BD02368F5
:1022000013F4805F0CD02B4AD2F8883023F040734F
:10221000216B0B43C2F88830236BB3F1807F3FD032
:10222000236813F4005F0CD0224AD2F8883023F0E0
:102230004063616B0B43C2F88830636BB3F1006F8E
:1022400033D0236813F4804F0CD01A4AD2F8883068
:1022500023F04063A16B0B43C2F88830A36BB3F14A
:10226000006F2BD0236813F4004F0CD0114AD2F822
:10227000883023F04053E16B0B43C2F88830E36BA6
:10228000B3F1805F1FD0284603B0F0BDD36843F49C
:102290008013D360A2E7D36843F48013D360AEE722
:1022A000D36843F48013D360BAE7D36843F4801350
:1022B000D360C6E70010024000700040D36843F4CA
:1022C0008013D360CEE7D36843F48033D360DAE77A
:1022D000F0B583B0002362E085685E000324B4405B
:1022E00025EA0405CC68B4402C438460456825EA9F
:1022F0000C054C68C4F300149C402C4344605FE020
:10230000DD08083550F8254003F0070C4FEA8C0C27
:102310004FF00F0E0EFA0CFE24EA0E0E0C6904FAB2
:102320000CF444EA0E0440F8254060E0052400E087
:10233000002404FA0EF42C430CF1020C554D45F820
:102340002C40554CA568D44325EA02064F6817F483
:10235000801F01D042EA05064F4DAE60ED6804EAE9
:1023600005064F6817F4001F01D042EA05064A4DE2
:10237000EE606D6804EA05064F6817F4003F01D06F
:1023800042EA0506444D6E602D682C404E6816F4F6
:10239000803F01D042EA05043F4A146001330A68D5
:1023A00032FA03F474D04FF0010C0CFA03FC1CEA6F
:1023B0000202F3D04C6804F00304013C012C8BD9D9
:1023C0004C6804F00304032C0CD0C4685D004FF08B
:1023D000030C0CFA05FC24EA0C0C8C68AC4044EAB3
:1023E0000C04C4604C6804F00304022C88D0046818
:1023F0004FEA430E4FF0030C0CFA0EFC24EA0C0CCF
:102400004C6804F0030404FA0EF444EA0C0404607B
:102410004C6814F4403FC1D0204C256E45F00105B6
:102420002566246E04F001040194019C4FEA930C8C
:102430000CF10205174C54F8255003F0030E4FEA37
:102440008E0E0F2404FA0EF425EA0405B0F1904F25
:102450003FF46EAF124CA04212D004F58064A0424B
:1024600010D004F58064A0420ED004F58064A04230
:102470000CD004F58064A0423FF458AF062458E71E
:10248000012456E7022454E7032452E7042450E7CA
:1024900003B0F0BD00000140000401400010024004
:1024A000000400480AB1816170478162704730B40E
:1024B000C46C056D6560446D14B1846DC56D656057
:1024C000446C04F01F0C012404FA0CF4056C6C60DD
:1024D000046863608368102B05D003689960036803
:1024E000DA6030BC704703689A600368D960F8E727
:1024F00003680C4A934213D80B49DBB2083B0B4AE2
:10250000A2FB0323426C22F003020A448264084ABD
:10251000C264C3F30413012202FA03F30365704794
:102520000449EAE70704024000080240CDCCCCCCC5
:1025300080080240200802400379074A1A449200AA
:102540004265064A8265013B03F01F03012202FA3D
:1025500003F3C365704700BF3F820010400902408B
:10256000002859D010B5044602682C4B9A423BD83B
:102570002B4B13442B49A1FB03131B099B00436402
:10258000294B0364022384F8253011686FF30E1180
:10259000A368E06803432069034360690343A069BB
:1025A0000343E0690343206A03430B43136020465F
:1025B000FFF79EFFA368B3F5804F20D0A36C22796C
:1025C0001A60E36C226D5A606368013B032B19D9D2
:1025D00000236365A365E3650020E063012384F8BD
:1025E000253084F8240010BD104B13440D49A1FB85
:1025F00003131B099B0043640D4B0364C2E70023D4
:102600006360DBE72046FFF797FF636D00221A60E7
:10261000A36DE26D5A60DFE70120704707040240B6
:10262000F8FFFDBFCDCCCCCC00000240F8FBFDBFD5
:102630000004024038B5044690F82400012841D037
:10264000012084F8240094F82500C0B2012804D0A9
:10265000002384F82430022038BD022084F82500AD
:102660000020E0632568286820F0010028602046EB
:10267000FFF71DFF236BD3B12268136843F00E03ED
:102680001360A36C1A6812F4803F03D01A6842F4F6
:1026900080721A60636D1BB11A6842F480721A600E
:1026A0002268136843F0010313600020D4E7226816
:1026B000136823F0040313602268136843F00A03CD
:1026C0001360DEE70220C7E7034690F82520D2B268
:1026D000022A09D00422C2630120012283F82520A6
:1026E000002283F82420704701680A6822F00E0255
:1026F0000A60816C0A6822F480720A6001680A68C4
:1027000022F001020A60426C02F01F01006C0122FB
:102710008A404260DA6C196D51605A6D42B111689D
:1027200021F4807111609A6DD96D51600020D4E759
:102730000020D2E708B590F82530DBB2022B09D093
:102740000423C363012380F82530002280F824206D
:10275000184608BD0268136823F00E031360026870
:10276000136823F001031360826C136823F48073F1
:102770001360436C03F01F02016C012393404B6014
:10278000C36C026D5A60436D33B11A6822F48072D3
:102790001A60836DC26D5A60012380F825300023D2
:1027A00080F82430836B13B198470020D1E70020D4
:1027B000CFE738B5036C196804682568436C03F0EB
:1027C0001F0304229A400A4215D015F0040F12D0BC
:1027D000236813F0200F03D1236823F00403236040
:1027E000436C03F01F02016C042393404B60036BA6
:1027F00003B1984738BD02229A400A421CD015F016
:10280000020F19D0236813F0200F06D1236823F09C
:102810000A032360012380F82530436C03F01F0274
:10282000016C022393404B60002380F82430C36A7C
:10283000002BDFD09847DDE7082202FA03F30B42B2
:10284000D8D015F0080FD5D0236823F00E032360ED
:10285000436C03F01F03016C012202FA03F34B6087
:10286000C26380F82520002380F82430436B002BBE
:10287000C0D09847BEE70000002836D13E4B1B6809
:1028800003F4C063B3F5806F08D03B4AD2F88030C0
:1028900023F48073C2F8803000207047364AD2F8A3
:1028A000803023F48073C2F88030136823F4C0634F
:1028B00043F400731360314B1B68322202FB03F3B5
:1028C0002F4AA2FB03239B0C013300E0013B2A4A61
:1028D000526912F4806F01D0002BF7D1264B5B694F
:1028E00013F4806F44D100207047B0F5007F08D00A
:1028F000214A136823F4C06343F48063136000200B
:1029000070471D4B1B6803F4C063B3F5806F08D09C
:10291000194AD2F8803043F48073C2F88030002026
:102920007047154AD2F8803043F48073C2F8803083
:10293000136823F4C06343F4007313600F4B1B68E8
:10294000322202FB03F30E4AA2FB03239B0C01334A
:1029500000E0013B084A526912F4806F01D0002B5D
:10296000F7D1054B5B6913F4806F03D100207047EA
:1029700003207047032070470070004008000020CB
:1029800083DE1B43024A936843F48043936070479D
:1029900000700040002807DB00F01F0240090123FF
:1029A0009340024A42F82030704700BF00E100E047
:1029B000002808DB0901C9B200F1604000F5614060
:1029C00080F80013704700F00F000901C9B2014BF5
:1029D0001954704714ED00E000B500F00700C0F195
:1029E000070CBCF1040F28BF4FF0040C031D062B8D
:1029F0000FD9C31E4FF0FF3E0EFA0CF021EA000182
:102A000099400EFA03FE22EA0E0241EA02005DF846
:102A100004FB0023EEE70000074AD36823F4E063D9
:102A20001B041B0C000200F4E060034343F0BF638F
:102A300043F40033D360704700ED00E010B5044666
:102A4000054BD868C0F30220FFF7C6FF01462046B9
:102A5000FFF7AEFF10BD00BF00ED00E008B5FFF7C7
:102A600099FF08BD0138B0F1807F0BD24FF0E02311
:102A70005861054AF02182F823100020986107224E
:102A80001A6170470120704700ED00E010B430304B
:102A90000B0A9B0003F00C03C45801F01F014FF018
:102AA0001F0C0CFA01FC24EA0C0CC2F384628A406D
:102AB0004CEA0202C2505DF8044B704710B4143067
:102AC0004B0E9B0003F00403C458C1F304514FF0B4
:102AD000070C0CFA01FC24EA0C0C8A404CEA0202B6
:102AE000C2505DF8044B704700B50C30C1F3015C77
:102AF00001F0010303EBC3030CEB830C50F82C3003
:102B000021F0024E2EF4601E23EA0E0311400B4307
:102B100040F82C305DF804FB30B583B000230193FE
:102B2000002800F001810446C36D13B323689A683E
:102B300012F0005F05D09A6822F0204222F03F0296
:102B40009A602268936813F0805F1FD1936823F026
:102B5000104323F03F0343F080539360734B1B6893
:102B60009B09734AA2FB03239B0901335B0001937A
:102B700009E0FEF7CBFB0023236684F85830D5E745
:102B8000019B013B0193019B002BF9D122689368C3
:102B900013F0805F40F09480E36D43F01003E36531
:102BA000236E43F0010323660120936813F00403AE
:102BB00000D00123E16D11F0100F40F0AE80002B2A
:102BC00040F0AB80E36D23F4817343F00203E365CF
:102BD000936813F0010F15D14FF0A0439A6812F0DB
:102BE000010200D00122534B9B6813F0010300D077
:102BF0000123134306D163684F498A6822F47C128B
:102C000013438B60627FE36B43EA4233E268134312
:102C1000A268134394F8242043EA0243012A51D0C6
:102C2000E26A22B102F47872216B0A4313432168ED
:102C3000CD68424A2A401A43CA602268136923F0C9
:102C40004063616B0B4313612268936813F00803C0
:102C500000D001232BBB237F94F83810490041EAB0
:102C60008331D36823F4804323F002030B43D36002
:102C7000236963B32268136943F4803313612268C4
:102C8000D2F8C0306FF30D0321690B43C2F8C03096
:102C900094F84030012B27D02268136923F00103F8
:102CA00013616369012B2FD02268136B23F00F038C
:102CB0001363E36D23F0030343F00103E36531E0A5
:102CC000002072E7A26A013A43EA4243A8E7226879
:102CD000136923F4803313612268D2F8C0306FF394
:102CE0000D03C2F8C030D3E721680B696FF38A0384
:102CF000626CA56C2A43E56C2A43256D2A43134375
:102D000043F001030B61CCE721680B6B23F00F0349
:102D1000226A013A13430B63CBE7E36D43F01003E0
:102D2000E365012003B030BD0120FBE7080000206F
:102D3000632D3E0500010050000300500740F0FFE6
:102D40000368186C7047704708B5806AFFF7FBFF8F
:102D500008BD7047F8B5044603681F685D689A4B64
:102D60009E6806F01F0617F0020F10D015F0020F34
:102D70000DD0C36D13F0100F03D1C36D43F4006386
:102D8000C365204600F0EAFE236802221A6017F0AD
:102D9000040F02D015F0040F05D117F0080F4DD025
:102DA00015F0080F4AD0E36D13F0100F03D1E36D57
:102DB00043F40073E3652368DA6812F4406F37D197
:102DC000824A934227D01A46934207D0092E25D82B
:102DD00040F22121F14011F0010F1FD0DA6812F406
:102DE000005F25D11A6812F0080F21D09A6812F0FE
:102DF000040F15D15A6822F00C025A60E36D23F4D7
:102E00008073E365E36D13F4805F11D1E36D43F0EC
:102E10000103E3650CE04FF0A042D5E7D268DEE79E
:102E2000E36D43F01003E365236E43F00103236673
:102E30002046FDF729FF23680C221A6017F0200FA7
:102E400002D015F0200F05D117F0400F5CD015F01F
:102E5000400F59D0E36D13F0100F03D1E36D43F42D
:102E60000053E3652368DA6C12F4C07F12D10121AC
:102E7000DA6812F4406F0FD10120544A93420DD00A
:102E80001A4693420DD066B1062E0AD0072E08D0FE
:102E9000D26807E00021EBE70020EEE74FF0A04208
:102EA000EFE7DA6851B312F0007F03D030B312F4C9
:102EB000005F23D1196811F0400F1FD012F4001FDA
:102EC0001CD19A6812F0080F10D15A6822F06002E3
:102ED0005A60E36D23F48053E365E36D13F4807F60
:102EE0000CD1E36D43F00103E36507E0E36D43F0CC
:102EF0001003E365236E43F001032366204600F0D0
:102F000029FE236860221A6017F0800F02D015F0A6
:102F1000800F2FD117F4807F02D015F4807F34D139
:102F200017F4007F02D015F4007F3AD117F0100F8C
:102F300019D015F0100F16D0E36B33B1002E3CD032
:102F4000214B9B6813F4604F0AD0E36D43F4806318
:102F5000E365236E43F0020323662046FFF7F9FE84
:102F6000236810221A6017F4806F02D015F4806F66
:102F70002ED1F8BDE36D43F48033E3652046FDF7C1
:102F800081FE236880221A60C4E7E36D43F40033B6
:102F9000E365204600F0E0FD23684FF480721A607C
:102FA000BEE7E36D43F48023E365204600F0D5FDE2
:102FB00023684FF400721A60B8E72368DB6813F0E7
:102FC000010FCDD0C1E700BF000300500001005049
:102FD000E36D43F48043E365236E43F00803236607
:102FE00023684FF480621A60204600F0B4FDC0E709
:102FF00008B50346806AC26D12F0500F30D1C36D20
:1030000043F40073C36503681A6812F0080F14D004
:10301000DA6812F4406F20D1DB6813F4005F1CD132
:10302000C36D23F48073C365C36D13F4805F14D143
:10303000C36D43F00103C3650FE0DB6813F0020FBB
:103040000BD1C36D23F48073C365C36D13F4805F2C
:1030500003D1C36D43F00103C365FDF715FE08BD41
:10306000C26D12F0100F04D1426D526B184690479A
:10307000F5E7FFF76EFEF2E708B5806AC36D43F02F
:103080004003C365036E43F004030366FFF761FE6C
:1030900008BD0000F0B583B00023019390F85830CC
:1030A000012B00F01C8204460D46012380F85830A5
:1030B0000068836813F0040F09D0E36D43F0200328
:1030C000E3650120002384F8583003B0F0BD0A689E
:1030D0004968FFF7DBFC2068836813F0040300D025
:1030E0000123866816F0080600D00126002B3ED189
:1030F000002E3CD1AA68B2F1004F6FD02968FFF7CB
:10310000DDFC2268536923F000435361696922683A
:10311000D368C3F3C1035B009940286904286AD0CF
:10312000603252F82070AB4B3B402F6807F0F84CF0
:1031300041EA0C010B4343F0004342F8203023687E
:103140002869AA69603353F8201021F080710A437E
:1031500043F82020236829692A7F012A48D0603358
:1031600053F8212022F00072324343F821202268D4
:10317000936813F0010F16D12B68E868D2F8B010ED
:10318000C3F3120621EA060100F018069248F04047
:103190000340C3F312030B43C2F8B030EA688F4B0D
:1031A0009A4200F08F802B688D4A134200F08F8185
:1031B0008C4A926802F0E0718B48834200F03E81B5
:1031C0008A48834200F03A818948834200F05C815A
:1031D0008848834200F06A81002073E70022296852
:1031E000FFF76CFC2268536943F0004353618DE79D
:1031F0004FF00076B3E7136E116EC1F384612B6854
:10320000C3F3120078BBC3F38463994233D02168BF
:103210004B6E4A6EC2F384622B68C3F3120078BB14
:10322000C3F384639A4233D021688B6E8A6EC2F3F3
:1032300084622B68C3F3120078BBC3F384639A42A1
:1032400033D02168CB6ECA6EC2F384622B68C3F39D
:10325000120078BBC3F384639A4288D1CB6E23F00B
:103260000043CB6683E793FAA3F313B1B3FA83F376
:10327000CBE72023C9E7136E23F000431366C6E7AC
:1032800093FAA3F313B1B3FA83F3CBE72023C9E78F
:103290004B6E23F000434B66C6E793FAA3F313B1DA
:1032A000B3FA83F3CBE72023C9E78B6E23F0004307
:1032B0008B66C6E793FAA3F313B1B3FA83F3CBE7B4
:1032C0002023C9E720682B68C3F3120626BB9A0E99
:1032D000013202F01F02092A8CBF00220122002ABB
:1032E00052D046BB990E0131890601F0F84176BBF8
:1032F0009F0E013707F01F070122BA401143AEBBF2
:103300009B0E013303F01F0303EB43031B0519431B
:10331000AA68FFF7D3FB46E793FAA3F24AB1B2FAE1
:1033200082F2013202F01F02092A8CBF0022012220
:10333000D5E72022F5E793FAA3F131B1B1FA81F193
:103340000131890601F0F841D1E72021F8E793FA2D
:10335000A3F24AB1B2FA82F2013202F01F024FF038
:10336000010C0CFA02F2C9E72022F5E793FAA3F365
:1033700043B1B3FA83F3013303F01F0303EB4303B9
:103380001B05C4E72023F6E7CEB9990E0131890663
:1033900001F0F84196BB9F0E013707F01F0701228D
:1033A000BA401143CEBB9B0E013303F01F0303EB66
:1033B00043031E3B1B0543F000731943A8E793FA30
:1033C000A3F1C9B1B1FA81F10131890601F0F841E7
:1033D000E0E700BF00F0FF03FFFF070000007F40B1
:1033E0000000088000030050000021C31000C090BE
:1033F000000052C7000084CB2021E5E793FAA3F236
:103400004AB1B2FA82F2013202F01F024FF0010C0F
:103410000CFA02F2C5E72022F5E793FAA3F35BB1B9
:10342000B3FA83F3013303F01F0303EB43031E3BA3
:103430001B0543F00073C0E72023F3E712F4000FED
:103440007FF4C2AE2368B3F1A04F01D0002039E66B
:1034500041F40001234A936823F0E073194391601B
:10346000214B1B689B09214AA2FB03239B090133C3
:1034700003EB43039B000193019B1BB1019B013BA9
:103480000193F9E700201DE612F0807F7FF4A0AEE3
:103490002268174B9A421CD041F08071114A936800
:1034A00023F0E0731943916000200BE612F4800FC3
:1034B00011D122680E4B9A420FD041F48003094982
:1034C0008A6822F0E07213438B600020FAE5002046
:1034D000F8E50020F6E50020F4E50020F2E5022002
:1034E000F3E500BF0003005008000020632D3E05F7
:1034F0000001005038B590F85830012B00F067817A
:1035000004460D46012380F858300068836813F0A4
:10351000040300D00123826812F0080200D00122C7
:103520007BBB72BB2968AB4B994262D06B68B3F12D
:10353000A07F00F0E28000F2D580B3F5400F00F0EC
:10354000DC80B3F1807F03D0B3F5000F40F0D18071
:10355000A14AFFF7C9FA2A68A04B9A4200F00481F9
:10356000E36D23F48023E36523684FF400721A604F
:103570002B7B012B00F00F812268536823F400732A
:1035800053602B68934A934200F00B812068C26815
:1035900002F01802182A00F013812969C268C2F3E8
:1035A000C102C2F10202520002F01E0221FA02FC24
:1035B000C26802F01802182A00F006816969C26820
:1035C000C2F3C102C2F10202520002F01E02D14057
:1035D000206820301B0D9B0003F00C03C25802F042
:1035E000F02241EA0C410A43C250002084F85800FE
:1035F00038BD6B68B3F1A07F48D011D8B3F5400F48
:1036000021D0B3F1807F4ED0B3F5000F5DD1C368F8
:1036100023F0FB4323F4800343F40003C3601EE064
:10362000B3F1C07F48D0B3F1E07F4ED1AA68C36840
:1036300023F0FB4323F4800302F0F84242F0E072EF
:103640001343C3600BE0AA68C36823F0FB4323F471
:10365000800302F0F84242F440021343C360226840
:10366000136A23F4E043A9690B431362E36D23F467
:103670008033E365236880221A602B7B012B2BD0DB
:103680002268536823F0800353607AE7AA68C3680E
:1036900023F0FB4323F4800302F0F84242F0A072CF
:1036A0001343C360DBE7C36823F0FB4323F48003C9
:1036B00043F08073C360D2E7C36823F0FB4323F475
:1036C000800343F0C073C360C9E7C36823F0FB43C2
:1036D00023F48003C360C2E72268536843F0800389
:1036E00053604EE7B3F1C07F3FF432AFB3F1E07FF8
:1036F00003D00022FFF7F8F92DE7384B99420DD09F
:10370000AB68C3F312021ABBC3F3846301229A406D
:10371000D0F8A4301343C0F8A4301CE7AB68C3F35F
:1037200012024AB9C3F3846301229A40D0F8A03050
:103730001343C0F8A0300EE793FAA3F333B1B3FA02
:1037400083F303F01F0301229A40EFE72023F8E7F9
:1037500093FAA3F333B1B3FA83F303F01F03012207
:103760009A40D5E72023F8E7E36D23F40033E365BF
:1037700023684FF480721A602B7B012B05D02268DE
:10378000536823F480735360FBE62268536843F464
:1037900080735360F5E62268536843F40073536006
:1037A000EFE629692068C268C2F3C102520001FA3B
:1037B00002FC6969C268C2F3C1025200914007E786
:1037C0002A694FEA820CF3E66969890000E7022062
:1037D0000EE700BF0000C07DFFFF8701FFFF17005D
:1037E00030B583B00023019303689A6812F0010F8B
:1037F00058D1044699682D4A114219D19A6822F08D
:10380000004222F03F0242F001029A60284B9B687E
:1038100013F4000F1CD0274B1B689B09264AA2FB00
:1038200003239B09013303EB43039B0001930CE04B
:10383000C36D43F01003C365036E43F001030366D9
:10384000012030E0019B013B0193019B002BF9D14A
:10385000FDF790FF054623681A6812F0010F1FD18B
:103860009A6812F0010F07D19A6822F0004222F004
:103870003F0242F001029A60FDF77CFF431B022BDE
:10388000E9D923681B6813F0010FE4D1E36D43F01D
:103890001003E365236E43F001032366012002E079
:1038A000002000E0002003B030BD00BF3F000080DA
:1038B0000003005008000020632D3E0538B5614B21
:1038C0009D6803689B6813F0040F40F0B6800446BF
:1038D00005F01F0590F85830012B00F0B08001234F
:1038E00080F85830FFF77CFF002840F0A280E36D9D
:1038F00023F4706323F0010343F48073E3652368CA
:10390000514A934257D01A46934200D01DB9E26DF6
:1039100022F48012E265E26D12F4805F4ED0226ED6
:1039200022F0060222661C221A60002384F8583016
:103930002268536823F01C035360A369082B40D00E
:103940002268536843F004035360E36B23B9226891
:10395000536843F01003536023683B4A934236D0C8
:103960001A46934207D0092D3ED840F22121E94062
:1039700011F0010F38D0DA6812F0007F11D0E26D3B
:1039800022F4405242F48052E265A269082A21D012
:103990005A6822F040025A602268536843F02003BC
:1039A00053602268936823F0004323F03F0343F001
:1039B0000403936042E04FF0A042A5E70022226694
:1039C000B1E72268536843F008035360BDE74FF046
:1039D000A042C6E75A6822F020025A602268536863
:1039E00043F040035360DCE7E16D41F48011E16591
:1039F000D26812F0007F21D0E26D22F4405242F4EE
:103A00008052E265A269082A09D05A6822F0400271
:103A10005A602268536843F0200353600EE05A68EE
:103A200022F020025A602268536843F0400353603A
:103A300004E0002384F8583000E0022038BD022062
:103A4000FCE700BF0003005000010050F8B5044639
:103A50003B4B9D680068806810F0040F6CD10E46E7
:103A6000174605F01F0594F85830012B66D0012346
:103A700084F85830092D05D840F22123EB4013F08B
:103A8000010F04D1002384F85830012055E020466E
:103A9000FFF7A6FE00284BD1E36D23F4706323F0FB
:103AA000010343F48073E3652368264A934239D0C7
:103AB0001A46934200D01DB9E36D23F48013E365E9
:103AC000E36D13F4805F30D0236E23F0060323668A
:103AD000636D1D4ADA62636D1C4A1A63636D1C4A8A
:103AE0005A6323681C221A60002384F85830226825
:103AF000536843F0100353602268D36843F0010316
:103B0000D36021683B4632464031606DFEF792FD3E
:103B10002268936823F0004323F03F0343F004033B
:103B200093600AE04FF0A042C3E700232366CFE78B
:103B3000002384F8583000E00220F8BD0220FCE7A2
:103B40000003005000010050F12F0008492D00082B
:103B50007930000870477047704770477047000021
:103B600090F85820012A7FD010B49DB0034601225E
:103B700080F858200022189219920068B0F1A04FE6
:103B800039D000220192019A002A37D0926812F0AF
:103B9000040200D00122806810F0040F54D1002AE2
:103BA00052D10A68002A32D0304CA26822F4604216
:103BB000486893F838C040EA4C300243A2604FF0A6
:103BC000A042906810F0010000D00120284A9268BD
:103BD00012F0010200D00122024341D1234CA2681D
:103BE00022F4716222F00F020868896801430A43D7
:103BF000A26000202DE01E4A0192C4E7DA6D42F077
:103C00002002DA65002283F85820012024E01749B9
:103C10008A6822F460428A604FF0A042916811F0F5
:103C2000010100D00121124A926812F0010200D075
:103C300001220A4316D10D498A6822F4716222F0EA
:103C40000F028A60002004E0DA6D42F02002DA659B
:103C50000120002283F858201DB05DF8044B704706
:103C60000020F6E70020F4E7022070470003005030
:103C70000001005003689A6912F0020F01D000227F
:103C80009A6203689A6912F0010F03D19A6942F0AF
:103C900001029A61704710B4019CC1F3090141EA25
:103CA00002411943214321F0004102685368640D29
:103CB00004F4806444F07F7444F4583444F47F7412
:103CC00044F0030423EA04030B4353605DF8044B00
:103CD00070472DE9F041044603689E6916F010060E
:103CE0007CD00D4690461022DA61002637462368C4
:103CF000986910F0200F30D17FBBB5F1FF3FF6D0AF
:103D0000FDF738FDA0EB0800A84201D8002DEED148
:103D100021684B6803F4804394F84220D2B288694A
:103D200010F4004F02D00BB9202A0ED123689B69F2
:103D300013F0200FDBD1FDF71DFDA0EB08001928C3
:103D4000F4D946F020060127D1E74B6843F48043BD
:103D50004B60FDF70FFD8046E8E70FB92022DA61DE
:103D600046F0040601252268936913F4807F05D08C
:103D700046F001064FF48071D161012513F4806F84
:103D800006D046F0080622684FF48061D161012513
:103D900013F4007F24D046F0020623684FF400722B
:103DA000DA6101252046FFF765FF2268536823F09A
:103DB000FF7323F48B3323F4FF7323F00103536069
:103DC000636C33436364202384F84130002384F818
:103DD000423084F840302846BDE8F0810025C2E733
:103DE000002DF8D0DEE770B504460D461646236870
:103DF0009B6913F0020F22D1324629462046FFF775
:103E000068FFF0B9B5F1FF3FF1D0FDF7B3FC801BBF
:103E1000A84201D8002DEAD123689B6913F0020F54
:103E2000E5D1636C43F020036364202384F84130C0
:103E3000002384F8423084F84030012000E0002064
:103E400070BD0120FCE72DE9F8430546884617467A
:103E50001E46DDF820902B689C6938EA04040CBFEC
:103E600001230023BB4227D14A4631462846FFF7AB
:103E700030FF20BBB6F1FF3FEDD0FDF77BFCA0EBA0
:103E80000900B04201D8002EE5D12B689B6938EAC1
:103E900003030CBF01230023BB42DCD16B6C43F056
:103EA00020036B64202385F84130002385F84230DD
:103EB00085F84030012000E00020BDE8F8830120B3
:103EC000FBE700002DE9F04182B0044690461D4614
:103ED000089E099F194B00934FF08073EAB2FFF7D9
:103EE000DAFE3A4631462046FFF77DFFF8B9012D4C
:103EF0000ED123685FFA88F29A6200973346002257
:103F000080212046FFF79FFFA8B902B0BDE8F081ED
:103F100023684FEA18229A623A4631462046FFF754
:103F200062FF30B923685FFA88F29A62E5E7012000
:103F3000EBE70120E9E70120E7E700BF0020008070
:103F40002DE9F04182B0044690461D46089E099F27
:103F5000184B00930023EAB2FFF79DFE3A46314624
:103F60002046FFF740FFF8B9012D0ED123685FFA14
:103F700088F29A6200973346002240212046FFF7DC
:103F800062FFA8B902B0BDE8F08123684FEA1822A9
:103F90009A623A4631462046FFF725FF30B923683A
:103FA0005FFA88F29A62E5E70120EBE70120E9E792
:103FB0000120E7E70020008070B504460D46164654
:103FC00004E023689B6913F0200F12D023689B69DB
:103FD00013F0200F1BD1324629462046FFF779FE09
:103FE000B8B9FDF7C7FB801BA842EAD8002DEDD178
:103FF000E7E7636C43F020036364202384F84130D7
:10400000002384F8423084F84030012000E0002092
:1040100070BD0120FCE700285FD010B5044690F881
:104020004130002B48D0242384F8413022681368A3
:1040300023F0010313606368226823F07063136147
:104040002268936823F400439360E368012B38D01F
:10405000A368226843F404439360E368022B36D0DC
:104060002268536823F4006353602268536843F066
:10407000007343F4004353602268D36823F4004381
:10408000D360236962691343A169226843EA01236B
:10409000D360E369216A22680B43136022681368C6
:1040A00043F00103136000206064202384F8413052
:1040B000206384F8420010BD80F84030FDF7DAF943
:1040C000B1E7A368226843F400439360C5E7226820
:1040D000536843F400635360C7E7012070472DE93C
:1040E000F04F83B00E46BDF834A00E9D90F84110FD
:1040F000C9B2202940F0BB800446904699460C9BEB
:10410000CBB1BAF1000F16D090F84030012B00F07F
:10411000B2804FF0010B80F840B0FDF72BFB074653
:10412000009019235A464FF400412046FFF78BFEBA
:1041300030B101209CE04FF400736364012097E0EC
:10414000212384F84130402384F842300023636403
:104150000C9A6262A4F82AA06363019700954B460B
:10416000424631462046FFF7ADFE70B9638D9BB2E3
:10417000FF2B0FD9FF222285002300934FF080737D
:1041800031462046FFF787FD21E0002384F84030C8
:1041900058466DE0628D92B22285002300934FF065
:1041A0000073D2B231462046FFF775FD0FE0628DF5
:1041B00092B22285002300934FF00073D2B23146B1
:1041C0002046FFF768FD638D9BB2002B33D03A4643
:1041D00029462046FFF707FE00284ED1626A236871
:1041E00012789A62636A01336362638D9BB2013B0A
:1041F0009BB26385238D013B9BB22385628D92B276
:10420000002AE0D0002BDED100972B46002280212F
:104210002046FFF718FE90BB638D9BB2FF2BC6D9DB
:10422000FF222285002300934FF080733146204601
:10423000FFF731FDC7E73A4629462046FFF7BCFEA7
:10424000F8B923682022DA6121684B6823F0FF73F4
:1042500023F48B3323F4FF7323F001034B6084F8C2
:104260004120002384F8423084F8403000E00220EE
:1042700003B0BDE8F08F0220FAE70120F8E7012043
:10428000F6E70120F4E700002DE9F04F83B00E4679
:10429000BDF834A00E9D90F84110C9B2202940F01D
:1042A000BC800446904699460C9BCBB1BAF1000FF6
:1042B00016D090F84030012B00F0B3804FF0010B86
:1042C00080F840B0FDF756FA0746009019235A4689
:1042D0004FF400412046FFF7B6FD30B101209DE0CC
:1042E0004FF400736364012098E0222384F8413086
:1042F000402384F84230002363640C9A6262A4F87D
:104300002AA06363019700954B46424631462046FA
:10431000FFF716FE70B9638D9BB2FF2B0FD9FF22FA
:104320002285444B00934FF0807331462046FFF7BF
:10433000B2FC21E0002384F8403058466EE0628DE4
:1043400092B222853B4B00934FF00073D2B23146BC
:104350002046FFF7A0FC0FE0628D92B22285002379
:1043600000934FF00073D2B231462046FFF793FC22
:10437000638D9BB2002B34D000972B460022042182
:104380002046FFF760FD00284DD123685A6A636A12
:104390001A70636A01336362228D013A92B22285F8
:1043A000638D9BB2013B9BB26385638D9BB2002BF7
:1043B000DED0002ADCD100972B4680212046FFF773
:1043C00042FD90BB638D9BB2FF2BC5D9FF22228596
:1043D000002300934FF0807331462046FFF75BFCCB
:1043E000C6E73A4629462046FFF7E6FDF8B92368B6
:1043F0002022DA6121684B6823F0FF7323F48B33AA
:1044000023F4FF7323F001034B6084F84120002361
:1044100084F8423084F8403000E0022003B0BDE868
:10442000F08F0220FAE70120F8E70120F6E70120EB
:10443000F4E700BF002400802DE9F04385B01D465D
:104440000023039390F84130DBB2202B40F08980A9
:1044500006468846914603689B6913F4004F40F076
:10446000828090F84030012B7FD0012380F84030CB
:10447000242380F841300023436441E0C8F309035A
:1044800043F0007343F4005343E033689C69C4F382
:1044900040149B69C3F30013C4B9BBB9B5F1FF3F26
:1044A000F3D0FDF767F9C01BA84201D8002DECD16D
:1044B000202386F84130736C43F02003736400239B
:1044C00086F84030012005B0BDE8F08333689B6971
:1044D00013F0100F2AD000972B46002220213046DF
:1044E000FFF7B1FC002844D133681022DA61336849
:1044F0002022DA61039B01330393039B4B4526D2B1
:10450000F368012BBAD0C8F3090343F0007343F4F6
:10451000205332685360FDF72DF9074633689C69D4
:10452000C4F340149B69C3F30013B5E700972B460F
:10453000002220213046FFF786FCC0B932682023D4
:10454000D36186F84130002386F84030BBE786F817
:104550004120736C13437364002386F840300120BC
:10456000B1E70220AFE70220ADE70220ABE7012070
:10457000A9E70120A7E7034690F84120D2B2202AFC
:1045800023D190F84020012A21D0012280F8402038
:10459000242280F841200068026822F001020260B3
:1045A0001868026822F48052026018680268114399
:1045B000016019680A6842F001020A60202283F84B
:1045C0004120002083F840007047022070470220FD
:1045D0007047034690F84120D2B2202A21D190F8AA
:1045E0004020012A1FD0012280F84020242280F898
:1045F00041200068026822F0010202601868026827
:1046000022F4706242EA0122026019680A6842F0EC
:1046100001020A60202283F84120002083F8400034
:1046200070470220704702207047000030B4026AD1
:10463000036A23F0010303624468836923F480332F
:1046400023F073030D681D4322F002028B681343AD
:104650001C4A90420FD002F5006290420BD002F546
:104660004062904207D002F58062904203D002F58A
:104670008062904205D123F00803CA681A4322F0F1
:104680000403104A90420FD002F5006290420BD012
:1046900002F54062904207D002F58062904203D05A
:1046A00002F58062904205D124F440744A692243A5
:1046B0008C691443446085614A684263036230BC7C
:1046C000704700BF002C014030B4036A026A22F434
:1046D000807202624468C26922F4803222F073025E
:1046E0000D68154323F400738A6843EA0223184ACD
:1046F000904203D002F50062904206D123F4006399
:10470000CA6843EA022323F48063114A90420FD01F
:1047100002F5006290420BD002F54062904207D051
:1047200002F58062904203D002F58062904207D188
:1047300024F440524C6942EA04128C6942EA04149F
:104740004460C5614A68C263036230BC704700BF01
:10475000002C014030B4036A026A22F480520262E3
:104760004468C26922F0807222F4E6420D6842EA8F
:10477000052223F400538D6843EA0533174DA84200
:1047800003D005F50065A84206D123F40043CD68A7
:1047900043EA053323F48043104DA8420FD005F5BA
:1047A0000065A8420BD005F54065A84207D005F585
:1047B0008065A84203D005F58065A84207D124F49E
:1047C000404C4C694CEA841C8C694CEA841444606B
:1047D000C2614A680264036230BC7047002C014029
:1047E00030B4036A026A22F4803202624468026DC5
:1047F00022F4803222F070020D68154323F4003356
:104800008A6843EA02430F4A90420FD002F50062E1
:1048100090420BD002F54062904207D002F58062D0
:10482000904203D002F58062904204D124F4803497
:104830004A6944EA0224446005654A688264036266
:1048400030BC7047002C014030B4036A026A22F485
:10485000801202624468026D22F0807222F4E0420B
:104860000D6842EA052223F400138D6843EA0553DC
:104870000F4DA8420FD005F50065A8420BD005F5F5
:104880004065A84207D005F58065A84203D005F52C
:104890008065A84204D124F480244D6944EA85242B
:1048A000446002654A68C264036230BC704700BF5E
:1048B000002C014010B4036A046A24F0010404626D
:1048C000846924F0F00C4CEA021223F00A030B4333
:1048D000826103625DF8044B704710B4036A046A96
:1048E00024F010040462846924F4704C4CEA02320F
:1048F00023F0A00343EA0113826103625DF8044BD5
:104900007047836823F4401323F070030B4343F094
:10491000070383607047000090F83D30DBB2012B45
:1049200032D1022380F83D300268D36843F001039E
:10493000D3600368174A934218D0B3F1804F15D063
:10494000A2F59432934211D002F5806293420DD0C9
:1049500002F59632934209D002F54062934205D0A7
:104960001A6842F001021A600020704799680A4AEA
:104970000A40062A0AD0B2F5803F09D01A6842F0F0
:1049800001021A6000207047012070470020704724
:1049900000207047002C014007000100704770475D
:1049A000704770477047704770B505460368DE680A
:1049B0001C6914F0020F10D016F0020F0DD06FF02A
:1049C00002021A610123037703689B6913F0030F46
:1049D0007CD0FFF7E6FF00232B7714F0040F12D0F2
:1049E00016F0040F0FD02B686FF004021A61022337
:1049F0002B772B689B6913F4407F6DD02846FFF717
:104A0000D0FF00232B7714F0080F12D016F0080FF8
:104A10000FD02B686FF008021A6104232B772B68E4
:104A2000DB6913F0030F5ED02846FFF7BAFF0023BF
:104A30002B7714F0100F12D016F0100F0FD02B6838
:104A40006FF010021A6108232B772B68DB6913F4CF
:104A5000407F4FD02846FFF7A4FF00232B7714F0A8
:104A6000010F02D016F0010F4BD114F4025F02D0F7
:104A700016F0800F4DD114F4807F02D016F0800F15
:104A80004FD114F0400F02D016F0400F51D114F066
:104A9000200F02D016F0200F53D114F4801F02D043
:104AA00016F4801F55D114F4001F02D016F4001F15
:104AB00057D114F4800F02D016F4800F59D114F49A
:104AC000000F02D016F4000F5BD170BDFFF768FF36
:104AD0002846FFF767FF7EE72846FFF761FF284675
:104AE000FFF760FF8DE72846FFF75AFF2846FFF7DC
:104AF00059FF9CE72846FFF753FF2846FFF752FF70
:104B0000ABE72B686FF001021A612846FFF747FFF9
:104B1000ABE72B686FF402521A61284600F095FB50
:104B2000A9E72B686FF480721A61284600F08EFBAB
:104B3000A7E72B686FF040021A612846FFF733FFA2
:104B4000A5E72B686FF020021A61284600F07CFB75
:104B5000A3E72B686FF480121A61284600F077FBF8
:104B6000A1E72B686FF400121A61284600F070FB71
:104B70009FE72B686FF480021A61284600F069FBFA
:104B80009DE72B686FF400021A61284600F062FB73
:104B90009BE700000368304A90420ED0B0F1804F8E
:104BA0000BD0A2F59432904207D002F58062904279
:104BB00003D002F59632904203D123F070034A6885
:104BC0001343254A90421AD0B0F1804F17D0A2F576
:104BD0009432904213D002F5806290420FD002F5D9
:104BE000963290420BD002F54062904207D002F517
:104BF0008062904203D002F58062904203D123F498
:104C00004073CA68134323F080034A691343036067
:104C10008B68C3620B6883620F4B98420FD003F519
:104C2000006398420BD003F54063984207D003F528
:104C30008063984203D003F58063984201D10B69E9
:104C4000036301234361036913F0010F03D0036978
:104C500023F0010303617047002C014060B310B5DD
:104C6000044690F83D3013B3022384F83D302146CA
:104C700051F8040BFFF78EFF012384F8483084F8C5
:104C80003E3084F83F3084F8403084F8413084F876
:104C9000423084F8433084F8443084F8453084F856
:104CA000463084F8473084F83D30002010BD80F84D
:104CB0003C30FCF739FCD7E70120704760B310B5F2
:104CC000044690F83D3013B3022384F83D3021466A
:104CD00051F8040BFFF75EFF012384F8483084F895
:104CE0003E3084F83F3084F8403084F8413084F816
:104CF000423084F8433084F8443084F8453084F8F6
:104D0000463084F8473084F83D30002010BD80F8EC
:104D10003C30FFF743FED7E70120704730B4036A09
:104D2000026A22F0100202624468826922F08072F4
:104D300022F4E6420D6842EA052223F020038D6842
:104D400043EA0513174DA84203D005F50065A842B4
:104D500006D123F08003CD6843EA051323F0400316
:104D6000104DA8420FD005F50065A8420BD005F5FF
:104D70004065A84207D005F58065A84203D005F537
:104D80008065A84207D124F4406C4C694CEA840C3D
:104D90008C694CEA8404446082614A6882630362DD
:104DA00030BC7047002C014038B590F83C30012BE6
:104DB00000F0958004460D46012380F83C30142A0B
:104DC00000F28880DFE802F00B8686861F868686E2
:104DD00034868686488686865D868686710000686B
:104DE000FFF724FC2268936943F00803936122686B
:104DF000936923F0040393612268936929690B4343
:104E00009361002067E00068FFF788FF22689369DC
:104E100043F4006393612268936923F48063936190
:104E200022689369296943EA01239361002052E0D3
:104E30000068FFF749FC2268D36943F00803D36197
:104E40002268D36923F00403D3612268D3692969F6
:104E50000B43D36100203EE00068FFF77BFC226833
:104E6000D36943F40063D3612268D36923F4806378
:104E7000D3612268D369296943EA0123D361002001
:104E800029E00068FFF7ACFC2268136D43F00803CB
:104E900013652268136D23F0040313652268136DF4
:104EA00029690B431365002015E00068FFF7CCFC6F
:104EB0002268136D43F4006313652268136D23F4B5
:104EC000806313652268136D296943EA0123136522
:104ED000002000E00120002384F83C3038BD02208F
:104EE000FCE710B4846824F47F4C42EA03220A43AE
:104EF00042EA0C0282605DF8044B704790F83C3047
:104F0000012B00F08F8010B50446012380F83C305F
:104F1000022380F83D3002689068434B0340936061
:104F20000B68702B55D031D8502B6CD01FD8402B2C
:104F30000AD1CA6849682068FFF7BCFC4021206894
:104F4000FFF7DFFC002029E068D8202B03D00AD827
:104F50000BB1102B05D119462068FFF7D2FC0020B9
:104F60001CE001201AE0302BF5D0012016E0602B68
:104F70000AD1CA6849682068FFF7AFFC6021206841
:104F8000FFF7BFFC002009E0012007E0B3F5005F58
:104F90002CD00AD8B3F5805F42D10020012384F8D9
:104FA0003D30002384F83C3010BD204A9342D2D0DB
:104FB00007D8B3F1101FCED0103A9342CBD00120C6
:104FC000ECE71B4A9342C6D030329342C3D0012053
:104FD000E4E7CB684A6889682068FFF782FF2268A7
:104FE000936843F0770393600020D7E7CB684A6863
:104FF00089682068FFF775FF2268936843F480434F
:1050000093600020CAE7CA6849682068FFF752FC2D
:1050100050212068FFF775FC0020BFE70120BDE7A5
:105020000120BBE7022070478800CEFF300010004F
:105030004000100001F01F014FF0010C0CFA01FCC0
:10504000036A23EA0C030362036A8A401343036280
:105050007047000010B5044610293CD8DFE801F085
:10506000093B3B3B1F3B3B3B263B3B3B2D3B3B3B01
:10507000340090F83E30DBB2013B18BF0123002B17
:1050800040F08E80102979D8DFE801F02C7878780C
:10509000687878786C78787870787878740090F898
:1050A0003F30DBB2013B18BF0123E8E790F8403006
:1050B000DBB2013B18BF0123E1E790F84130DBB2DE
:1050C000013B18BF0123DAE790F84230DBB2013B25
:1050D00018BF0123D3E790F84330DBB2013B18BF80
:1050E0000123CCE7022384F83E3001222068FFF739
:1050F000A1FF23682D4A93420FD002F5006293422C
:105100000BD002F54062934207D002F580629342D1
:1051100003D002F58062934203D15A6C42F40042FC
:105120005A642368214A93422CD0B3F1804F29D08E
:10513000A2F59432934225D002F58062934221D0A9
:1051400002F5963293421DD002F54062934219D087
:105150001A6842F001021A60002022E0022384F85B
:105160003F30C2E7022384F84030BEE7022384F8D0
:105170004130BAE7022384F84230B6E7022384F8CC
:105180004330B2E799680A4A0A40062A0AD0B2F5C3
:10519000803F09D01A6842F001021A60002000E046
:1051A000012010BD0020FCE70020FAE7002C0140A0
:1051B0000700010090F83C20012A40D030B403469B
:1051C000012280F83C20022280F83D2000684268DD
:1051D00084681C4DA84203D005F50065A84203D1A0
:1051E00022F470024D682A4322F0007222F070020D
:1051F0000D682A4342601A681248824212D0B2F106
:10520000804F0FD0A0F5943082420BD000F5806023
:10521000824207D000F59630824203D000F540600C
:10522000824204D124F080048968214391600122E4
:1052300083F83D20002083F83C0030BC70470220FA
:10524000704700BF002C014070477047704770479F
:10525000704770477047026852E8003F23F0C00370
:1052600042E800310029F6D1026802F1080353E850
:10527000003F23F40003083242E800310029F3D153
:105280002023C0F888307047026852E8003F23F4BA
:10529000907342E800310029F6D1026802F1080358
:1052A00053E8003F23F0805323F00103083242E823
:1052B00000310029F1D1C36E012B06D02023C0F8A4
:1052C0008C300023C36643677047026852E8003F92
:1052D00023F0100342E800310029F6D1EEE708B5CB
:1052E000026852E8003F23F0400342E80031002901
:1052F000F6D12023C0F8883000238367FBF7DEFC5B
:1053000008BD70477047704738B5846AD4F8882064
:10531000D4F88C5023689B6813F0800F01D0212AA9
:1053200010D023689B6813F0400F01D0222D10D0BD
:10533000D4F8903043F01003C4F890302046FFF7C3
:10534000E2FF38BD0023A4F856302046FFF783FF64
:10535000E7E70023A4F85E302046FFF795FFE7E774
:1053600008B5806A0023A0F85E30FFF7CCFF08BDC7
:1053700070B504460268D3691068916840F60F0C56
:1053800013EA0C0F0DD113F0200F10D010F0200FE6
:1053900002D111F0805F0AD0636F93B32046984723
:1053A0002FE09D4D0D402DD19C4E30422AD1E56E0F
:1053B000012D00F0C08013F4801F03D011F4800F82
:1053C00040F06C8113F0800F07D010F0800F40F098
:1053D0006C8111F4000F40F0688113F0400F03D08E
:1053E00010F0400F40F0688113F4000F03D010F06C
:1053F000804F40F0658113F0807F02D00028C0F21A
:10540000638170BD13F0010F09D010F4807F06D0C6
:1054100001261662D4F890203243C4F8902013F08D
:10542000020F0BD011F0010F08D02268022616627D
:10543000D4F8902042F00402C4F8902013F0040F36
:105440000BD011F0010F08D0226804261662D4F8A0
:10545000902042F00202C4F8902013F0080F0BD005
:1054600010F0200F00D13DB1226808251562D4F854
:1054700090202A43C4F8902013F4006F0CD010F051
:10548000806F09D022684FF400651562D4F890202F
:1054900042F02002C4F89020D4F89020002AB0D026
:1054A00013F0200F09D010F0200F02D111F0805F0F
:1054B00003D0636F0BB120469847D4F8902023683F
:1054C0009B6813F0400F02D112F0280F2CD0204619
:1054D000FFF7DAFE23689B6813F0400F20D02268A4
:1054E00002F1080353E8003F23F04003083242E88A
:1054F00000310029F3D1D4F880306BB1484A9A6367
:10550000D4F88000FDF716F900283FF47AAFD4F8FC
:105510008000836B984774E72046FFF7F4FE70E73E
:105520002046FFF7F0FE6CE72046FFF7ECFE002375
:10553000C4F8903065E713F0100F3FF43CAF10F063
:10554000100F3FF438AF1023136223689B6813F0E9
:10555000400F67D0D4F880100A6853689BB2002BC4
:105560004AD0B4F85C00984246D9A4F85E300B6883
:105570001B6813F0200F32D1226852E8003F23F459
:10558000807342E800310029F6D1226802F1080355
:1055900053E8003F23F00103083242E800310029BC
:1055A000F3D1226802F1080353E8003F23F04003DF
:1055B000083242E800310029F3D12023C4F88C30AE
:1055C0000023E366226852E8003F23F0100342E81C
:1055D00000310029F6D1D4F88000FDF775F80223D8
:1055E0002367B4F85C10B4F85E309BB2C91A89B274
:1055F0002046FBF74FFB04E7B4F85C1099427FF4B8
:1056000000AF136813F0200F3FF4FBAE02232367B3
:105610002046FBF73FFBF4E60100001020010004E8
:1056200061530008B4F85C10B4F85E309BB2C91A3C
:1056300089B2B4F85E309BB2002B3FF4E2AE002991
:105640003FF4DFAE226852E8003F23F4907342E853
:1056500000300028F6D1226802F1080353E8003F29
:1056600023F0805323F00103083242E80030002881
:10567000F1D12023C4F88C300023E36663672268ED
:1056800052E8003F23F0100342E800300028F6D132
:10569000022323672046FBF7FDFAB2E64FF480139E
:1056A0001362204600F044FCABE6A36F002B3FF4EE
:1056B000A8AE20469847A4E62046FFF710FEA0E6D5
:1056C000204600F037FC9CE6204600F032FC98E6CD
:1056D00008B5806A01230367C36E012B02D0FFF770
:1056E00011FE08BDB0F85C104908FBF7D3FAF8E7E3
:1056F00008B50346806A1B681B6813F0200F29D188
:105700000023A0F85E30026852E8003F23F4807363
:1057100042E800310029F6D1026802F1080353E89B
:10572000003F23F00103083242E800310029F3D1A1
:10573000026802F1080353E8003F23F040030832F7
:1057400042E800310029F3D12023C0F88C30C36E29
:10575000012B07D000230367C36E012B0CD0FFF78A
:10576000D0FD08BD026852E8003F23F0100342E874
:1057700000310029F6D1EDE7B0F85C10FBF78AFAAA
:10578000EFE7000070B5044683680269134342697D
:105790001343C2691343016808688B4A02401A43E5
:1057A0000A602268536823F44053E1680B43536056
:1057B000A1692268854B9A4201D0236A19439368F4
:1057C00023F06E4323F430630B4393602268D36A63
:1057D00023F00F03616A0B43D36223687C4A934230
:1057E00023D07C4A934234D07B4A93424AD07B4AAE
:1057F000934259D0754A934268D0102273498B4224
:1058000000F09580E069B0F5004F00F0D280082AE2
:1058100000F24F81DFE812F01201340110014D0156
:1058200037014D014D014D013A0102F55842D2F8C0
:10583000882002F00302032A09D8DFE802F00204FC
:105840005C060122DAE70422D8E70822D6E7102214
:10585000D4E702F5E632D2F8882002F00C020C2AD6
:105860000ED8DFE802F0070D0D0D090D0D0D4A0DE4
:105870000D0D0B000022C1E70422BFE70822BDE79F
:105880001022BBE702F5E432D2F8882002F03002A1
:10589000202A34D004D8A2B3102A34D10422ADE790
:1058A000302A32D10822A9E702F5E232D2F8882064
:1058B00002F0C002802A2AD004D852B3402A2AD14A
:1058C00004229BE7C02A28D1082297E702F5C832B4
:1058D000D2F8882002F44062B2F5006F1FD005D8DC
:1058E000FAB1B2F5806F1ED1042287E7B2F5406F9E
:1058F0001BD1082282E7022280E702227EE70222F1
:105900007CE700227AE7102278E7102276E702226D
:1059100074E7002272E7102270E710226EE702227D
:105920006CE700226AE7102268E7102266E7082A7F
:1059300000F2AF80DFE802F008AD3BAD38ADADADB1
:1059400005004FF4004004E0FCF72CFB002800F0B9
:10595000A280626A224B33F81220B0FBF2F3656832
:1059600005EB4501994200F29880B3EB053F00F248
:105970009680002633463146FBF7A0F8090241EA3B
:10598000106100026B08C0182A46334641F100013D
:10599000FBF794F8A0F54072124B9A4200F2818016
:1059A0002368D860304662E0FCF7B6F9CEE70E48CF
:1059B000CFE7082A77D8DFE802F0193905763C7678
:1059C00076761D00084815E0F369FFCF008000409F
:1059D000003801400044004000480040004C0040B6
:1059E00090720008FFFC0F000024F400FCF7DAFAC4
:1059F00000285AD0626A324B33F81230B0FBF3F011
:105A00006268530803EB4003B3FBF2F3A3F1100108
:105A10004FF6EF7291424AD89AB222F00F02C3F3C6
:105A2000420313432268D360002020E0FCF7CCFA45
:105A3000DEE7FCF771F9DBE7224803E0FCF7B2FA96
:105A4000002838D0626A1E4B33F81230B0FBF3F0F6
:105A5000636800EB5300B0FBF3F0A0F110024FF6C7
:105A6000EF739A4229D8236880B2D86000200123BE
:105A7000A4F86A30A4F8683000236367A36770BD98
:105A8000FCF7A2FADCE7FCF747F9D9E74FF400404E
:105A9000D8E70120EBE70020E9E70120E7E7012054
:105AA000E5E70120E3E70120E1E70020DFE701204F
:105AB000DDE70120DBE70020D9E70120D7E700BFC1
:105AC000907200080024F400836A13F0080F06D0D7
:105AD0000268536823F40043816B0B435360836A6D
:105AE00013F0010F06D00268536823F40033C16A33
:105AF0000B435360836A13F0020F06D002685368A9
:105B000023F48033016B0B435360836A13F0040F5B
:105B100006D00268536823F48023416B0B43536023
:105B2000836A13F0100F06D00268936823F4805341
:105B3000C16B0B439360836A13F0200F06D0026899
:105B4000936823F40053016C0B439360836A13F052
:105B5000400F0AD00268536823F48013416C0B4352
:105B60005360436CB3F5801F0BD0836A13F0800F32
:105B700006D00268536823F40023C16C0B435360C2
:105B800070470268536823F4C003816C0B43536071
:105B9000EBE72DE9F84305460E4617469946DDF832
:105BA00020802B68DC6936EA04040CBF0124002441
:105BB000BC4236D1B8F1FF3FF3D0FBF7DBFDA0EBE1
:105BC0000900404530D8B8F1000F2FD02B681A6873
:105BD00012F0040FE5D0802EE3D0402EE1D0DA6938
:105BE00012F0080F11D1DA6912F4006FD9D04FF416
:105BF00000621A622846FFF747FB2023C5F8903061
:105C0000002385F8843003200CE008241C62284619
:105C1000FFF73AFBC5F89040002385F88430012057
:105C200000E00020BDE8F8830320FBE70320F9E74C
:105C30002DE9F04182B01E46D0F88830202B5AD191
:105C400004460D469046002959D00AB9012053E078
:105C50000023C0F890302123C0F88830FBF78AFD7C
:105C60000746A4F85480A4F85680A368B3F5805F73
:105C700002D04FF0000816E0236943B34FF000084C
:105C800011E02023C4F88830032035E038F8023BC7
:105C90002268C3F308039362B4F8562092B2013A23
:105CA00092B2A4F85620B4F856309BB293B1009645
:105CB0003B46002280212046FFF76BFF0028E0D101
:105CC000002DE3D015F8012B23689A62E4E7A8467B
:105CD0000025E8E700963B46002240212046FFF7DA
:105CE00058FF18B92023C4F8883005E02023C4F8F1
:105CF0008830032000E0022002B0BDE8F0810120DE
:105D0000FAE730B583B004460023C0F89030FBF7C3
:105D100031FD05462268126812F0080F10D1236881
:105D20001B6813F0040F28D12023C4F88830C4F86E
:105D30008C300020E066206784F8840003B030BD1A
:105D40006FF07E430093034600224FF4001120467B
:105D5000FFF71FFF0028E2D0226852E8003F23F03F
:105D6000800342E800310029F6D12023C4F88830AE
:105D7000002384F884300320E0E76FF07E43009333
:105D80002B4600224FF480012046FFF702FF002837
:105D9000CAD0226852E8003F23F4907342E80031F1
:105DA0000029F6D1226802F1080353E8003F23F0EE
:105DB0000103083242E800310029F3D12023C4F85E
:105DC0008C30002384F884300320B7E778B310B513
:105DD0000446D0F888300BB32423C4F888302268F6
:105DE000136823F001031360A36AE3B92046FFF7A9
:105DF000C9FC012811D02268536823F490435360F2
:105E00002268936823F02A0393602268136843F0A2
:105E1000010313602046FFF774FF10BD80F8843043
:105E2000FBF7E0FBD8E72046FFF74EFEDEE7012058
:105E30007047000010B5044613468165A0F85C2049
:105E40000022C0F890202222C0F88C20D0F88020B8
:105E5000AAB12149D162D0F8802020491163D0F83D
:105E600080201F495163D0F8802000219163016890
:105E7000826D2431D0F88000FCF7DCFB20BB236965
:105E800043B1226852E8003F43F4807342E8003196
:105E90000029F6D1226802F1080353E8003F43F0DD
:105EA0000103083242E800310029F3D1226802F1EF
:105EB000080353E8003F43F04003083242E8003152
:105EC0000029F3D1002010BD1023C4F89030202306
:105ED000C4F88C300120F6E7F1560008D1560008CE
:105EE00009530008436E2BB90123A0F86A30A0F8CB
:105EF0006830704730B403689A68C2F342629968A8
:105F0000490F094D6B5CDB00084C615C93FBF1F3BE
:105F1000A0F86A30AB5CDB00A25C93FBF2F3A0F864
:105F2000683030BC704700BFB0720008A87200082B
:105F300070477047704790F88430012B18D00123C8
:105F400080F884302423C0F8883003681A68196800
:105F500021F00101196022F000520023436601681C
:105F60000A602022C0F8882080F8843018467047E4
:105F70000220704738B590F88430012B1DD00446BC
:105F8000012380F884302423C0F8883003681D681A
:105F90001A6822F001021A600268936823F06043D5
:105FA00019439160FFF79EFF23681D602023C4F80A
:105FB0008830002084F8840038BD0220FCE738B522
:105FC00090F88430012B1DD00446012380F88430E2
:105FD0002423C0F8883003681D681A6822F0010283
:105FE0001A600268936823F0606319439160FFF7B9
:105FF00079FF23681D602023C4F88830002084F8CE
:10600000840038BD0220FCE7D0F88C30202B1FD153
:1060100010B50446F1B10AB9012010BD0123C366D1
:1060200000230367FFF706FF0028F6D1E36E012B7C
:1060300001D00120F1E7236810221A62226852E899
:10604000003F43F0100342E800310029F6D1E4E7B5
:10605000022070470120E0E7034AD2F8883043F479
:106060007003C2F88830704700ED00E010B50346B9
:106070000C4A0D490D48006840B10C4800680344C3
:10608000521A934206D8094A136010BD0748084CBB
:106090000460F2E700F0DEFA0C2303604FF0FF30FB
:1060A000F3E700BF0080002000040000000400208F
:1060B000B805002010B586B004468DF8171064238B
:1060C0000322C0210948FEF7B7F90028F7D164235D
:1060D0000293012301930DF1170200922246C02181
:1060E0000248FDF7FCFF06B010BD00BF6C020020A7
:1060F00010B586B00446059164230322C0210948E7
:10610000FEF79AF90028F7D1642302930123019343
:1061100005AA00922246C0210248FEF7B5F806B053
:1061200010BD00BF6C0200202DE9F84F80460C46E0
:10613000674B984249D8674B984238D9FAF7EAF941
:1061400002460B465CA1D1E90001FAF787FBFAF79A
:1061500095FC05282ED910F0010F2CD001302AE033
:10616000760001357F2E04DC08FB06F2594B9A427B
:10617000F6D92D01374608FB06F0FAF7CBF90246AF
:106180000B464DA1D1E90001FAF768FBFAF776FC5E
:1061900010F0010F00D0013000FB07F708FB07F7F4
:1061A0004D4B9F424ED802304FF0000A12E00025BE
:1061B0000126D7E7062008FB00F2474B9A4244D855
:1061C000023001260025AA4604E0012600254FF0F2
:1061D0000C0A042000F10077043FFF0106FB00F0E9
:1061E00008FB00F0FAF796F935A3D3E90023FAF794
:1061F00035FB80468946FAF719FC0646FAF79AF904
:1062000002460B4640464946FAF746F8804689461C
:106210002DA3D3E90023FAF7F7F9FAF72FFC834609
:10622000B8B1FAF777F942464B46FAF717FB002266
:106230002A4BFAF733F8FAF721FCB0F5801F09D39F
:10624000274807E04FF0000AC4E701260025AA46C8
:10625000C0E723484FEACB1BBBFBF0F303EBC616AA
:10626000A6F5007600FB13BB030A23706070C6F32B
:106270000143A370330AE3702671000B00F0F000B5
:10628000CBF30343184360714FEA1B23A37184F8D7
:1062900007B000232372012262725544EDB2C7F3A6
:1062A00001421544A5723A0AE27227736373A3731D
:1062B000E373BDE8F88F00BF00000000A3E1C14117
:1062C00000000000FC64724100000000FEFF2F414E
:1062D00080D1F00868780400FF45C3230000E03F48
:1062E000FFFF0F0010B5002421460020FFF700FF3C
:1062F00010F0800FF8D1FF212C4B19700320FFF70D
:10630000D9FE00210F20FFF7D5FE00211820FFF74E
:10631000D1FE00212A20FFF7CDFE01212B20FFF71F
:10632000C9FE00212F20FFF7C5FE00213020FFF716
:10633000C1FE00213120FFF7BDFE00213220FFF712
:10634000B9FE01213320FFF7B5FE00213720FFF70A
:10635000B1FE00213820FFF7ADFE00213920FFF704
:10636000A9FE00213A20FFF7A5FE01213B20FFF7FF
:10637000A1FE00213F20FFF79DFE00214020FFF7F6
:1063800099FE00214120FFF795FE4F211020FFF7D5
:1063900091FE5F211120FFF78DFE6F211220FFF784
:1063A00089FE1221B720FFF785FE10BD04040020EE
:1063B00010B584B00C466946FFF7B6FE94B1012CC7
:1063C0001FD100242EE004F110036B4404F11A00E5
:1063D00013F8101CC0B2FFF76DFE0134072CF2DD7C
:1063E0000A240CE00024F9E704F110036B4404F1E3
:1063F000220013F8101CC0B2FFF75CFE01340C2C15
:10640000F2DD2021B120FFF755FE04B010BD04F1EC
:1064100010036B4404F1220013F8101CC0B2FFF704
:1064200049FE0134072CF2DD0A240AE004F11003CE
:106430006B4404F12A0013F8101CC0B2FFF73AFEB7
:1064400001340C2CF2DDDCE708B501238340044A5B
:10645000117821EA030111700320FFF72BFE08BD1C
:10646000040400200000000008B51149022000F0DB
:10647000B1F8104B0CA1D1E90001C3E900010023E0
:106480000D4A13600D4A13600D4B0E4A1A600E4BF5
:106490000A221A8014225A801E229A802822DA8028
:1064A00008BD00BFAFF300809A9999999999D93F97
:1064B000D0720008100400200C0400200804002002
:1064C0002404002098BC14001C040020B0F5006FC8
:1064D0000AD3A0F500639BB2C3F3C703054A107843
:1064E000984200D818467047C0F5FF6307339BB247
:1064F000F2E700BF6C04002008B50349022000F059
:1065000069F8FFF7EFFE08BDDC72000810B504461D
:106510000649022000F05EF800212046FFF748FF00
:1065200001212046FFF744FF10BD00BFE8720008BC
:1065300008B50549022000F04DF80020FFF784FF60
:106540000120FFF781FF08BDF87200080123024A0D
:106550001370024A137070476E0400206B04002011
:1065600010B50C464FF47A738AB201460348FFF720
:106570005FFB034B00221A70204610BD4001002033
:106580006A04002000B595B00E4B1A885988988887
:10659000DB8803930290019100920B4B1B780B4A0E
:1065A000402104A800F088F804A8F9F719FE014674
:1065B00004A8FFF7D5FF064B00221A7015B05DF84E
:1065C00004FB00BF1C0400206D04002004730008BD
:1065D0006C04002000B593B003460091074A4021A7
:1065E00002A800F069F802A8F9F7FAFD014602A82E
:1065F000FFF7B6FF13B05DF804FB00BF2873000877
:106600000D488546FFF728FD0C480D490D4A00232B
:1066100002E0D458C4500433C4188C42F9D30A4A57
:106620000A4C002301E013600432A242FBD300F0C5
:1066300017F8FAF771FDFEE7008000200000002047
:106640005C0000207C73000860000020B80500207A
:10665000FEE70000014B1868704700BF0C000020E7
:1066600070B50D4D0D4C641BA4100026A64209D137
:106670000B4D0C4C00F000FE641BA4100026A6423B
:1066800005D170BD55F8043B98470136EEE755F843
:10669000043B98470136F2E77473000874730008EE
:1066A000747300087873000802440346934200D1D3
:1066B000704703F8011BF9E70CB430B5184B0C1EFA
:1066C0001D689DB008DA8B232B604FF0FF301DB0A2
:1066D000BDE8304002B070474FF40273ADF814309B
:1066E0004FF000031B9314BF04F1FF3323460493C0
:1066F00007934FF6FF7302900690ADF81630209A7C
:1067000021AB02A92846019300F068F8431CBCBFE6
:106710008B232B60002CDAD0029B00221A70D6E764
:106720000C0000202DE9F0478E681F46BE420B6822
:1067300082460C4690462DD8B1F90C2012F4906F89
:1067400026D06569096905EB4505A3EB010905EB51
:10675000D5757B1C4B446D109D4238BF1D465305BB
:1067600027D5294600F000FB064660B321694A465A
:1067700000F07AFBA38923F4906343F08003A381A4
:10678000266165614E44A5EB09052660A5603E467D
:10679000BE4200D93E4620683246414600F01AF912
:1067A000A3689B1BA3602368334423600020BDE8DB
:1067B000F0872A4600F082FB06460028E0D12169D6
:1067C000504600F0A9FB0C23CAF80030A38943F01F
:1067D0004003A3814FF0FF30E9E700002DE9F04FBF
:1067E00098468B891B069DB007460D46144610D56A
:1067F0000B6973B9402100F0B7FA2860286130B9FD
:106800000C233B604FF0FF301DB0BDE8F08F4023FC
:106810006B610023099320238DF82930CDF80C807B
:106820003023DFF89C818DF82A304FF00109234690
:106830009A4613F8012B0AB1252AF9D1BAEB040BB9
:106840000BD05B46224629463846FFF76BFF0130E6
:1068500000F0A780099A5A4409929AF80030002B58
:1068600000F09F8000234FF0FF32CDE905230AF1AD
:10687000010A049307938DF853301A935446052266
:1068800014F8011B4E48F9F7B3FC049AD8B9D006A6
:1068900044BF20238DF85330110744BF2B238DF8BC
:1068A00053309AF800302A2B15D0079A544600200E
:1068B0004FF00A0C214611F8013B303B092B4BD914
:1068C000B0B1079214E0A0EB080309FA03F31343F5
:1068D0000493A246D2E7039B191D1B680391002B6A
:1068E000BBBF5B4242F0020207930793B8BF04921A
:1068F00023782E2B0AD163782A2B32D1039B1A1DC1
:106900001B68039243EAE37302340593DFF8C0A0E7
:10691000217803225046F9F76BFC38B1049BA0EBB9
:106920000A004022824013430134049314F8011BEF
:1069300024488DF828100622F9F75AFC002836D092
:10694000214B1BBB039B073323F00703083303933F
:10695000099B334409936AE70CFB02320C46012081
:10696000A8E700230134059319464FF00A0C20468E
:1069700010F8012B303A092A03D9002BC6D0059113
:10698000C4E70CFB012104460123F0E703AB0093AD
:106990002A460E4B04A93846AFF30080421C064637
:1069A000D6D1AB895B063FF52DAF09982CE703AB39
:1069B00000932A46054B04A9384600F095F8EDE708
:1069C00037730008417300080000000025670008C5
:1069D0003D730008884210B501EB020402D98442DD
:1069E000234607D8431EA14208D011F8012B03F813
:1069F000012FF8E7024401468A4200D110BD13F886
:106A0000014D02F8014DF7E7704770472DE9F04757
:106A1000164698468A680B69DDF820909342B8BF05
:106A20001346336091F8432007460C460AB1013300
:106A300033602368990642BF3368023333602568A8
:106A400015F0060506D104F1190AE36832689B1AAD
:106A5000AB4226DC94F843302268003B18BF012388
:106A600092062BD404F1430241463846C847013010
:106A70001ED02368226903F00603042B02BFE568D9
:106A80003368ED1AA3680CBF25EAE575002593422B
:106A9000C4BF9B1AED1800261A34B5421AD1002043
:106AA00008E00123524641463846C847013003D129
:106AB0004FF0FF30BDE8F0870135C6E7E1185A1CFA
:106AC000302081F84300224494F8451082F84310A6
:106AD0000233C7E70123224641463846C847013002
:106AE000E6D00136D9E700002DE9FF470F7E0C9E66
:106AF000782F914680460C469A4601F1430207D80A
:106B0000622F0AD8002F00F0D180582F00F0B880F3
:106B100004F1420684F842703AE0A7F16303152BB2
:106B2000F6D801A151F823F0816B0008956B00089D
:106B3000116B0008116B0008116B0008116B000845
:106B4000956B0008116B0008116B0008116B0008B1
:106B5000116B0008936C0008BF6B00084D6C0008B7
:106B6000116B0008116B0008B56C0008116B000870
:106B7000BF6B0008116B0008116B0008556C000812
:106B800033681A1D1B68326004F1420684F84230F3
:106B900001239CE033682068191D3160060601D589
:106BA0001D6803E04506FBD5B3F90050002D03DA5C
:106BB0002D236D4284F8433058480A2311E02168A0
:106BC0003368080653F8045B02D4490648BFADB2E7
:106BD0006F2F5248336014BF0A230823002184F822
:106BE00043106668A660002E05DB21682E4321F065
:106BF000040121604BD01646B5FBF3F103FB11579E
:106C0000C75D06F8017D2F46BB420D46F4D9082B1F
:106C10000BD12368DF0708D5236961689942DEBF7D
:106C2000302306F8013C06F1FF36921B2261CDF8B5
:106C300000A04B4603AA21464046FFF7E7FE01307D
:106C40004AD14FF0FF3004B0BDE8F087236843F02D
:106C5000200323603248782784F845702368316820
:106C60001F0651F8045B02D45F0648BFADB2316025
:106C7000D90744BF43F0200323601DB11023ADE7C3
:106C80002648E9E7236823F020032360F6E7164649
:106C9000BDE7336825686169181D30602E061B68E2
:106CA00001D5196002E06806FBD519800023236135
:106CB0001646BCE733681A1D32601E686268002100
:106CC0003046F9F795FA08B1801B6060636823616C
:106CD000002384F84330AAE72369324649464046F8
:106CE000D0470130ADD023689B0713D4E068039BE5
:106CF0009842B8BF1846A6E70123324649464046A7
:106D0000D04701309DD00135E36803995B1AAB424F
:106D1000F2DCEBE7002504F11906F5E748730008FB
:106D20005973000870B50F4E0C463168054611B90D
:106D300000F0B4F830602146284600F0AFF8431C5C
:106D400003D14FF0FF34204670BDC41C24F003046F
:106D5000A042F8D0211A284600F0A0F80130F2D164
:106D6000EFE700BFAC0500202DE9F843CD1C25F06E
:106D7000030508350C2D38BF0C25002D064601DB18
:106D8000A94204D90C2333600020BDE8F883DFF862
:106D9000D48000F077F8D8F800301C4644BB294670
:106DA0003046FFF7BFFF431C044658D1D8F80040D7
:106DB0002746002F43D1002C4BD02368394630465C
:106DC00004EB030900F06AF8814542D121686D1A8D
:106DD00029463046FFF7A6FF01303AD023682B44FE
:106DE0002360D8F800305A6862BBC8F800700FE022
:106DF0002268521B20D40B2A17D96119A34225609F
:106E000018BF5960636808BFC8F8001062514B6032
:106E1000304600F03DF804F10B00231D20F0070080
:106E2000C21A1CBF1B1AA350AFE76268A3420CBF73
:106E3000C8F800205A60EBE723466468AEE73C469A
:106E40007F68B6E71A465B68A342FBD10023536014
:106E5000DEE70C233360304600F01AF894E7056053
:106E6000D6E700BFB00500200A44914200F1FF338D
:106E700000D1704710B511F8014B03F8014F914252
:106E8000F9D110BD0148FFF7BFBD00BFA805002024
:106E90000148FFF7BABD00BFA805002038B5064D70
:106EA0000023044608462B60FFF7E0F8431C02D19C
:106EB0002B6803B1236038BDB40500202DE9F041F3
:106EC000074614460D4621B9BDE8F0411146FFF7CB
:106ED0004BBF2AB900F020F825462846BDE8F081CE
:106EE00000F064F88442064602D8B4EB500FF4D8A0
:106EF00021463846FFF738FF804608B94546ECE79B
:106F0000B4422246294628BF3246FFF7ADFF294644
:106F1000384600F001F8F1E738B50546002941D0C0
:106F200051F8043C0C1F002BB8BFE418FFF7AAFF70
:106F30001D4A136833B9636014602846BDE83840C1
:106F4000FFF7A6BFA34208D9206821188B4201BFD2
:106F500019685B6809182160EDE71A465B680BB198
:106F6000A342FAD911685018A0420BD120680144FD
:106F7000501883421160E0D118685B685360084480
:106F80001060DAE702D90C232B60D6E720682118BD
:106F90008B4204BF19685B68636004BF09182160F5
:106FA0005460CAE738BD00BFB005002051F8043C6A
:106FB000181F002BBCBF0B58C01870472DE9F047B5
:106FC000089D0E4604460F46002B4AD194468C4538
:106FD000B2FA82F260D942B1C2F12003974020FA9E
:106FE00003F30CFA02FC1F4394404FEA1C4E1FFAB5
:106FF0008CF6B7FBFEF1230C0EFB117743EA074337
:1070000001FB06F098420AD91CEB030301F1FF379C
:1070100080F01581984240F21281023963441B1AB4
:10702000A4B2B3FBFEF00EFB103344EA034400FBB2
:1070300006F6A6420AD91CEB040400F1FF3380F0E7
:107040000081A64240F2FD806444023840EA0140DB
:10705000A41B00211DB1D4400023C5E90043BDE8B5
:10706000F0878B4205D90DB1C5E900010021084622
:10707000F5E7B3FA83F1002946D1B34202D3824245
:1070800000F2F580841A66EB030201201746002DFA
:10709000E5D0C5E90047E2E7002A40F09380A1EB84
:1070A0000C034FEA1C471FFA8CFE0121B3FBF7F6D5
:1070B00007FB1630230C43EA00430EFB06F0984210
:1070C00008D91CEB030306F1FF3802D2984200F204
:1070D000D08046461B1AA4B2B3FBF7F007FB10336F
:1070E00044EA03440EFB00FEA64508D91CEB040449
:1070F00000F1FF3302D2A64500F2B6801846A4EB99
:107100000E0440EA0640A5E7C1F120078B4022FAB1
:1071100007FC4CEA030C06FA01FE20FA07F426FAF3
:1071200007F344EA0E0400FA01F84FEA1C404FEA64
:107130001449B3FBF0FE1FFA8CF600FB1E3349EA3C
:1071400003430EFB06F9994502FA01F20BD91CEB39
:1071500003030EF1FF3A80F08580994540F282806A
:10716000AEF1020E6344A3EB0909A4B2B9FBF0F33C
:1071700000FB139944EA094403FB06F6A64208D92A
:107180001CEB040403F1FF3068D2A64266D9023B2F
:10719000644443EA0E40A41BA0FB02E6B4427346DB
:1071A000B14652D34FD05DB1B8EB030264EB090492
:1071B00004FA07F722FA01F31F43CC40C5E9007433
:1071C00000214CE7C2F1200120FA01F30CFA02FC85
:1071D00026FA01F1964033434FEA1C471FFA8CFE12
:1071E000B1FBF7F007FB1016190C41EA064100FB52
:1071F0000EF68E4204FA02F408D91CEB010100F1EC
:10720000FF382DD28E422BD902386144891B9BB2A4
:10721000B1FBF7F607FB161143EA014306FB0EF13B
:10722000994208D91CEB030306F1FF3814D29942A6
:1072300012D9023E63445B1A46EA004136E73946FA
:10724000EDE6184602E7F045ADD2BEEB020366EB71
:107250000C060138B146A6E74646ECE7034698E738
:107260004046D3E7D6467EE76444023847E70846FF
:107270000DE7023E63442DE7F8B500BFF8BC08BC3B
:107280009E467047F8B500BFF8BC08BC9E467047E4
:10729000010002000400060008000A000C001000B3
:1072A00020004000800000010804020408010101E0
:1072B00001010103070100000000000001020304B6
:1072C0000000000000000000010203040607080996
:1072D000737175656F7720696E69740073796E7468
:1072E0006820696E6974000073796E746820736534
:1072F000742066726571000073796E7468206F6E19
:10730000000000001B5B3364444D5020563D256C4B
:107310007520543D257520433D257520443D257538
:1073200020523D25750A00001B5B32644C4F4720FC
:1073300025752025730A00232D302B2000686C4C06
:10734000006566674546470030313233343536379D
:1073500038394142434445460030313233343536C2
:0C73600037383961626364656600000024
:08736C00748EFF7F0100000098
:04737400590B0008A9
:04737800310B0008CD
:10737C0001000000100000000024F40010000020A8
:10738C000000000070040020D804002040050020FC
:10739C0000000000000000000000000000000000E1
:1073AC0000000000000000000000000000000000D1
:1073BC0000000000000000000000000000000000C1
:0C73CC00000000000000000000000000B5
:040000050800660188
:00000001FF
